:047245000100033011
:106CB600AF50055074D02FF582E4341DF583E59965
:106CC600F022D3E5309400E52F94002290000FE0E7
:036CD60064032232
:03000300025AA9F5
:0B5AA900C0E0C083C082C0D075D008F0
:105AB400852E82852D83E493FF201404C4540FFFA4
:105AC400430FF08F80C284D28500C2870000D28742
:105AD400007580FF7580FEC284C28500C287000005
:105AE400D287007580FF30140CC214052EE52E7089
:095AF40006052D8002D214D2A88F
:095AFD00D0D0D082D083D0E03279
:03000B00021BFFD6
:101BFF00C0E0C0F0C083C082C0D075D008758CD84B
:101C0F00758A92D28C1244B0126627E531D39400B4
:101C1F0040171531E53164056009E531640F600344
:101C2F00021E11126EFB021E11753114E54ED39474
:101C3F00004002154EE54FD394004002154FE53A90
:101C4F00D394004002153AE54BD394004002154B54
:101C5F00154CE54C12126B1E03001DD8011DB0026E
:101C6F001D88031D05041CEC051CD3061CBA071C9C
:101C7F00A1081C880900001E0ED3E52C9400E52B4B
:101C8F0094005003021E11E52C152C704D152B02DC
:101C9F001E11D3E5379400E53694005003021E1150
:101CAF00E537153770021536021E11D3E54894003B
:101CBF00E54794005003021E11E5481548700215C0
:101CCF0047021E11D3E54A9400E5499400500302E0
:101CDF001E11E54A154A70021549021E11D3E52A55
:101CEF009400E52994005003021E11E52A152A706D
:101CFF00021529021E117884E6FF7003021E11EFF0
:101D0F00B40105900524801BEFB40210126CC8407B
:101D1F002FE53015307002152F021E11EFB4030C92
:101D2F00900526E0F52FA3E0F5308028EFB40412DC
:101D3F00126CC8400BE53015307002152F021E11C2
:101D4F008012EF64057003021E11EFB4060C752F9D
:101D5F0002753058788406021E11EF640760030283
:101D6F001E11126CC8400BE53015307002152F0292
:101D7F001E1178847600021E11D3E5399400E538E0
:101D8F0094004008E539153970021538D3E53C94B5
:101D9F0000E53B9400406BE53C153C7002153B8021
:101DAF0061D3E5579400E55694004008E557155761
:101DBF0070021556D3E5559400E55494004043E561
:101DCF00551555700215548039D3E5359400E53417
:101DDF0094004008E535153570021534301523D3BE
:101DEF00E5339400E53294004018E5331533701253
:101DFF001532800EE551D3940040041551800075C3
:0D1E0F004C0AD0D0D082D083D0F0D0E03289
:03001300023D1893
:0D3D1800C0E0C0F0C083C082C0D075D010E4
:103D2500E545C394504003023DE8202403023DE8E5
:103D3500300C03023DE8E5A0540FF5587D077F01DF
:103D450012519B5067202364E545700DE558B40C6E
:103D550008201105D211023DE820034A201147121F
:103D65003DF350047F0180027F0F1271C890000F50
:103D7500E0FF64016012EFB40302800C90000FE0D5
:103D8500B40209123DF350047F80801290000FE0C9
:103D9500B4020E7D037F0712519B40057FA01200E0
:103DA50016754202D20390053CE0F53A7D087F0581
:103DB50012519B501A90002BE0B55807202304D2CE
:103DC500268020053EE53EAE3D700E053D800A0588
:103DD5003EE53EAE3D7002053D14F5828E83E55805
:033DE500F00545A1
:103DE800D0D0D082D083D0F0D0E0327D037F0712CC
:033DF800519B22BA
:0300230002670071
:10670000C0E0C083C082C0D075D018309819C2983C
:10671000E599B40A08126CB6755000800AE550C3BA
:1067200094905003126CB6309902C299D0D0D082A6
:05673000D083D0E0322F
:03003B0002485622
:0D485600C0E0C0F0C083C082C0D075D01893
:10486300C2CEE546C394104003024900202503024B
:104873004900300C03024900AFA07804EF0880011F
:1048830023D8FDF55953590F7D077F0212519B50D1
:1048930035202332E546700CE559B40C0720130488
:1048A300D213805920041920131690000FE0B4028C
:1048B3000F7F0A1271C87F80120016754202D2045C
:1048C30090053CE0F53A7D087F0512519B501A9004
:1048D300002BE0B55907202304D22880200540E5AA
:1048E30040AE3F700E053F800A0540E540AE3F7085
:0D48F30002053F14F5828E83E559F005465D
:0B490000D0D0D082D083D0F0D0E032C5
:104ED400E4F55AF55B755C1E755DFF855B82855A4A
:104EE40083E0F55E635EFFE55EF0E0655E600312FD
:104EF4007249635EFF855B82855A83E55EF0E065F7
:104F04005E6003127249055BE55B7002055AE55D5C
:104F1400155D7002155CD3E55D9400E55C9400506A
:104F2400BA75985A758921758845758DE775878096
:104F3400758CD8758AEF75C90275C808753D1E75DC
:104F44003E60753F1E7540B075B701D2A9D2E8D254
:0F4F5400AA75C64C75EEFF75FEFFD2AF126A014B
:014F6300222B
:0272490080FEC5
:106C9300202F0F90053AE0F54EE54ED394004012B5
:106CA30080F7302F0D90053AE0F54FE54FD3940070
:036CB30050F92273
:106C4B0030310AD215900024E04420800DC2157F0C
:106C5B0008127209900024E054DFF0FD7F247E00BF
:046C6B001266CA22C1
:103160008F6AE56A640170292030047F018056204F
:10317000300302325B12326C400302325B12327453
:10318000500C12325C30150302325B0232510232B3
:1031900011E56A640270202030047F02802720300D
:1031A0000302325B12327C400302325B126CD2703B
:1031B0000302325B02322BE56A6403600302325B76
:1031C0002030057F0302720930302412326C501F08
:1031D00012327C501A126CD26015123274500B7F6E
:1031E0000B1232842015740232517F0302325830A0
:1031F0003023123292501E7D017F0212519B4015E6
:103200007D017F0712519B500812325C20154C80C3
:10321000407F01804330301712329240127D017F8F
:103220000212519B5009126CD260047F0280293037
:1032300030297D017F0112519B5020126CD2701BEE
:103240007D017F0712519B500D7F0912328420159A
:103250000AD231026C4B7F0112721C227F0912725A
:103260001C900536E0F532A3E0F533227D017F01A5
:1032700012519B227D017F0712519B227D017F020B
:1032800012519B2212721C900536E0F532A3E0F534
:0A32900033227D017F0112519B22C1
:104F6400C2957FAA127209124ED47F0712665E5050
:104F74000512003E80031263ADD28C7F0812665E78
:104F8400500512457080FEC22B126B919000D1E047
:104F9400FF7C117D00125E9A12600D90000FE0B448
:104FA4000105122AC7801090000FE0FF640260041C
:104FB400EFB403031234FB123FBF301E11E54270FD
:104FC4000DE52754A060077FA01271C8C21E7D079B
:104FD4007F0512519B4002C200E552C3940A50BBA4
:104FE4003015B8E533453270B2C231126C4B80AB28
:104DAD00EF253EFFEE353DCF2401FDE43FFC22AF64
:104DBD005A7E00EF2403FDEE33FC22E53E255AF525
:104DCD0082E4353DF58322E540255AF582E4353FF1
:104DDD00F58322E56F256DF582E4356EF583E0FFF1
:104DED00E56F256DF582E4356EF58322E55A2402D3
:104DFD00FFE433FE22E56C2401FFE433FEC3E56DD1
:104E0D009FEE6480F874809822EF2540FFEE353FC9
:104E1D0022E55C2EF582E4355BF583E0FD227FF41F
:104E2D007E01126F6DE56C25E0F56C756D012275D7
:064E3D003D1E753E6022DF
:106F6D00EF1FAA0670011ED39400EA9400400BE4B3
:0A6F7D00FDEDC394C850E90D80F744
:016F870022E7
:10552F008F5BE55BB401197D017F0612519B500C17
:10553F009000B1E0FF7C0D7D00125E9A7884062208
:10554F00E55BB402131255A150439000B2E0FF7C0B
:10555F000D7D20125E9A8035E55BB404161255A1BD
:10556F00500C9000B4E0FF7C0D7D60125E9A788441
:10557F00760622E55BB403197D027F0612519B501C
:10558F000C9000B3E0FF7C0D7D40125E9A7884761C
:0A559F0001227D027F0612519B22BB
:10519B00BF0107900020E0FE8048BF02079000216E
:1051AB00E0FE803EBF0307900022E0FE8034BF0488
:1051BB0007900023E0FE802ABF0507900024E0FE45
:1051CB008020BF0607900025E0FE8016BF070790E2
:1051DB000026E0FE800CBF0807900027E0FE80024F
:1051EB00E4FEBD0103EE1322BD0204EEA2E122BDDB
:1051FB000304EEA2E222BD0404EEA2E322BD0504E9
:10520B00EEA2E422BD0604EEA2E522BD0704EEA247
:07521B00E622BD0802EE339C
:015222002269
:10201D00124E3C900100E0F55A124DC8E012126BC1
:10202D00204C0120810220B60320EB042120052144
:10203D005506218A0721BA0821E60900002210124F
:10204D004DC8A3E0B40A15E55A124DFBE545B50799
:10205D000BE4B506077D017F010221CE124DBCE5D3
:10206D00456D7001EC6003022210124DADC2297F47
:10207D00010221E3124DC8A3E0B40A15E55A124D31
:10208D00FBE545B5070BE4B506077D017F0202218F
:10209D00CE124DBCE5456D7001EC600302221012AD
:1020AD004DADC2297F020221E3124DC8A3E0B40A4F
:1020BD0015E55A124DFBE545B5070BE4B506077D51
:1020CD00017F030221CE124DBCE5456D7001EC6020
:1020DD0003022210124DADC2297F030221E3124DDE
:1020ED00C8A3E0B40A15E55A124DFBE545B5070B3B
:1020FD00E4B506077D017F040221CE124DBCE545F6
:10210D006D7001EC6003022210124DADC2297F04E7
:10211D000221E3124DC8A3E0B40A15E55A124DFB96
:10212D00E545B5070BE4B506077D017F050221CE18
:10213D00124DBCE5456D7001EC6003022210124D8D
:10214D00ADC2297F050221E3124DC8A3E0B40A15E3
:10215D00E55A124DFBE545B5070BE4B506077D01C4
:10216D007F060221CE124DBCE5456D7001EC60037A
:10217D00022210124DADC2297F060221E3124DC875
:10218D00A3E0B40A14E55A124DFBE545B5070AE480
:10219D00B506067D017F078028124DBCE5456D70A3
:1021AD0001EC705F124DADC2297F078029124DC819
:1021BD00A3E0B40A0F124DC8A3A3E070077D017F01
:1021CD0008025110124DBCE5456D7001EC703412D2
:1021DD004DADC2297F08021291124DC8A3A3E07024
:1021ED0022124DC8A3E024F96008147016E4FF0212
:1021FD0062747FF47E01126F6D7D5E7F021269D76E
:03220D0012457007
:0122100022AB
:101E1C00753F1E7540B0900108E0F55A124DD4E0A4
:101E2C0012126B1E4E011E86021EBE031EF6041FEE
:101E3C002E051F66061F9E071FD1082006090000ED
:101E4C00201C124DD4A3E0B40A13124DF9E546B58B
:101E5C00070BE4B506077D017F01021FE9AF5A129B
:101E6C004DBEE5466D7001EC600302201C124E164F
:101E7C00124DB4D2297F01022003124DD4A3E0B439
:101E8C000A13124DF9E546B5070BE4B506077D01BB
:101E9C007F02021FE9AF5A124DBEE5466D7001EC90
:101EAC00600302201C124E16124DB4D2297F02027E
:101EBC002003124DD4A3E0B40A13124DF9E546B534
:101ECC00070BE4B506077D017F03021FE9AF5A1229
:101EDC004DBEE5466D7001EC600302201C124E16DF
:101EEC00124DB4D2297F03022003124DD4A3E0B4C7
:101EFC000A13124DF9E546B5070BE4B506077D014B
:101F0C007F04021FE9AF5A124DBEE5466D7001EC1D
:101F1C00600302201C124E16124DB4D2297F04020B
:101F2C002003124DD4A3E0B40A13124DF9E546B5C3
:101F3C00070BE4B506077D017F05021FE9AF5A12B6
:101F4C004DBEE5466D7001EC600302201C124E166E
:101F5C00124DB4D2297F05022003124DD4A3E0B454
:101F6C000A13124DF9E546B5070BE4B506077D01DA
:101F7C007F06021FE9AF5A124DBEE5466D7001ECAB
:101F8C00600302201C124E16124DB4D2297F060299
:101F9C002003124DD4A3E0B40A12124DF9E546B554
:101FAC00070AE4B506067D017F078031AF5A124D52
:101FBC00BEE5466D7001EC7057124E16124DB4D240
:101FCC00297F078032124DD4A3E0B40A13124DF9C5
:101FDC00E546B5070BE4B506077D017F08025110F5
:101FEC00AF5A124DBEE5466D7001EC7023124E16C1
:101FFC00124DB4D2297F08021291124DD4A3A3E042
:10200C00700E124DD4A3E024F870057F0112627497
:01201C0022A1
:044B20008C5B8D5CC1
:104B2400055CE55C7002055B14F5828C83E0F9702A
:104B340003024BC7EF7005124E3C8009BF01067596
:104B44003F1E7540B0302946EF7007E965456002A5
:104B5400C322BF0107E965466002C322E4FEEEC337
:104B6400995029EF700F124E1EE53E2E124DCCE0E7
:104B74006D6002C322EF6401700F124E1EE5402ED9
:104B8400124DD8E06D6002C3220E80D2D3222029B8
:104B940033E4FEEEC3995029EF700F124E1EE53E2A
:104BA4002E124DCCE06D6016C322EF6401700F121B
:104BB4004E1EE5402E124DD8E06D6002C3220E80D9
:044BC400D2D322C363
:014BC80022CA
:061291008F5BAB05AA040F
:101297007D027F0712519B5011E55BB4050C8B82D1
:1012A7008A83E0640570030214FE7D017F071251F3
:1012B7009B5011E55BB4050C8B828A83E064067052
:1012C700030214FEC22AEB24FFF582EA34FFF583FA
:1012D700E0F55D8B828A83E0FFF55EA3E0F9F55FB9
:1012E700EF12126B130701130E02131503131C04DD
:1012F700132305132A061331071338080000133D7B
:10130700755C01D22A802F755C02D22A8028755C11
:1013170004D22A8021755C08D22A801A755C10D203
:101327002A8013755C20D22A800C755C40D22A80F3
:1013370005755C80D22AE924FE70030213FF24F8A6
:10134700605C24096003021411E55BB40105900099
:10135700208045E55BB40205900021803BE55BB446
:1013670003059000228031E55BB4040590002380DB
:1013770027E55BB40505900024801DE55BB40605F1
:101387009000258013E55BB407059000268009E5EA
:101397005B64087077900027E0455CF0806EE55B42
:1013A700B401059000208045E55BB402059000215B
:1013B700803BE55BB403059000228031E55BB40414
:1013C700059000238027E55BB40505900024801D68
:1013D700E55BB406059000258013E55BB40705902F
:1013E70000268009E55B64087022900027E0FFE58E
:1013F7005CF4FEEF5EF08014E55BB4050D8B828A2A
:1014070083E0FFD22F122C28C22AC22A202A0302E5
:1014170014FEE55BB40109900020E0FD7F208060A9
:10142700E55BB40209900021E0FD7F218052E55B76
:10143700B40309900022E0FD7F228044E55BB404F9
:1014470009900023E0FD7F238036E55BB405099012
:101457000024E0FD7F248028E55BB4060990002581
:10146700E0FD7F25801AE55BB40709900026E0FDC3
:101477007F26800CE55BB4080C900027E0FD7F27F2
:101487007E001266CA127067D2AF2029047F0180DE
:10149700027F0212721CA229922F126C93AD5DE497
:1014A700FF1269D7AD5EE4FF1269D7E55FB40104A7
:1014B7007D388007E55FB40A077D367F061269D756
:1014C700E55BB405031268347D077F0512519B5015
:1014D7000A200007C2307F031231607D017F0112AD
:1014E700519B4005C2301231607D017F0212519B32
:0714F7004005C23012316014
:0114FE0022CB
:025110008F5BB3
:10511200ED24FF922F126C93E55B12126B513B014F
:10512200514002514503514A04514F055154065111
:105132005907515E080000516490002080219000C0
:1051420021801C900022801790002380129000245E
:10515200800D90002580089000268003900027E0B3
:10516200F55CE55C6024755E01E4F55DE55C30E0CC
:1051720007AD5EE4FF1269D7E55CC313F55C055E1B
:10518200055DE55DC3940840E3227D187F02126944
:08519200D77D537F021269D79B
:01519A0022F2
:10665E00C2AFD284C285BF070BC28600E580A2E21C
:10666E00922A8019BF080BC28600E580A2E3922A07
:10667E00800BBF0508C28600E58013922AD286D20F
:05668E0085D2AFA22A35
:0166930022E4
:10490B00C229D22DE4FF125CC77D2E7F031269D71B
:10491B007D607F021269D77F031272093024FD205C
:10492B0024FDE5456407703B7E017F50124E3C8FA2
:10493B00828E837407F07D01E53E2D124DCCE5820E
:10494B0024FFF582E58334FFF583E0F9EF2DF58243
:10495B00E43EF583E9F00DBD08DED2297F647E00CD
:10496B00126F6D7F0812665E5043302995D22DE48D
:10497B00FF125CC77D607F021269D77D327F061202
:10498B0069D77D1E7F051269D7C22DE4FF125CC764
:10499B007C017D507B087F507E011258C37F08122B
:1049AB00665E50097F327E00126F6D80F07F647EF1
:0449BB0000126F6D0A
:0149BF0022D5
:02577C008F5A42
:10577E00900138E0F55BE55A7020E55B124DFBE5D4
:10578E00456F7001EE70547460255BF582E4341E33
:10579E00AF82F55D8F5E7F408024E55A6401703BD9
:1057AE00E55B124DFBE5466F7001EE702E74B02571
:1057BE005BF582E4341EAF82F55D8F5E7F101200C2
:1057CE0016855E82855D83E0FFA3E0FD1270B58FC6
:0B57DE005CE4FD124BC97F501271C843
:0157E900229D
:024BC9008D6BF2
:104BCB0075F020EF90028012125FAF8285836E8F9B
:104BDB006FE0F56CD394005003024C68E56C9410B5
:104BEB00507BE56B7014124E2B124E02506F124D10
:104BFB00E0124C69056D056D80EFE56B6401702A61
:104C0B00C201124E2B124E025053124DE0124C6940
:104C1B00302402800A30250C90000FE0B402057F8F
:104C2B00500271C8056D056D80DBE56B6402702D5C
:104C3B00C201C202124E2B124E025021124DE0A3A2
:104C4B00E0FD126864302402800A30250A90000FC0
:0D4C5B00E0B40203024253056D056D80DADE
:084C680022A3E0FD12686422A2
:100D2900855C82855B83A3A3E0FF855C82855B8309
:100D3900A3222430F58274003EF583EDF0AF62EF13
:100D49003395E0FEE55F2FF582E55E3EF58322E50A
:100D5900822406F582E43583F583E0FF127090ADB5
:100D690007AF63EF3395E0FEEF22A3A3E0FFE55C55
:100D79002404F582E4355BF583E022E55F2405F57B
:100D890082E4355EF583E022E55F2405F582E435EA
:100D99005EF583E0FFE55F2406F582E4355EF583C1
:100DA900E0228E69F56AAF68EF3395E0FEE5662FBC
:100DB900F582E5653EF583222455F582E4340AF58A
:100DC90083EFF0E56275F007A422AF60EF3395E099
:100DD900FEE56175F00890015812125FE5822FF562
:100DE90082E5833EF58322E5662405F582E43565CF
:100DF900F583E022E55E75F007A42454F582E43416
:100E09000AF58322A3A3A3E0FF8D828C83E58224C4
:100E190004F582E43583F583E022E55E75F007A4E5
:100E29002451F582E4340AF5832224E0F582740A18
:100E39003EF583E5822DF582E5833CF58322E55E67
:100E490075F007A42453F582E4340AF58322E55F9B
:100E59002405F582E4355EF583E0FFE55F2406F5B8
:100E690082E4355EF583E022E55E75F007A424523D
:100E7900F582E4340AF58322749F2562F582E4340D
:100E890000F58322746F2562F582E43400F583222C
:100E99002450F582E4340AF58322ECFF3395E0FE11
:100EA900EF25E0FFEE33FE75F02022E5602405F51D
:100EB90082E4355FF58322D3EF6480948022AB0707
:100EC900AA068B828A83A3A3A3E0FFEB2404F582FD
:100ED900E43AF583E0FD228F828E83A3A3A3E02267
:100EE900855F82855E83A3A322AB5DAD5AAF5CAEFD
:100EF9005B22FFE562FD3395E0FCE55F2DF582E5B8
:100F09005E3CF5832233CE33CE92E022A2E0CE13AB
:100F1900CE132275F00AA42DFDE5F03CFCE566220E
:100F2900E5602405F582E4355FF583E022E5627525
:100F3900F00890015802125FE55E75F007A4245588
:100F4900F582E4340AF583E022AB5AAD5DAF5CAEBD
:100F59005B22EF7C002563FDEC35628D82F58322EF
:100F6900A3A3E0FFAD5A22540FF5657808AF03AE8D
:100F790002EF08220564E564AE632275F0201212BF
:100F89005FE0FEA3E0FF22E0FAA3E0FB780CFFAEEE
:100F9900020822E0FCA3E0FD7804FFAE040822E584
:100FA900632561F582E43562F58322E5662DF582D4
:100FB900E5653CF58322E5662FF582E5653EF58317
:100FC900222431F5827400222480F58274023EAF16
:100FD90082222560F560E4355FF55F2285608285B0
:0D0FE9005F83228F828E83A3A3E0640A221F
:020556008F5ABA
:10055800C22AE4F542D223D22D125CC77D4B7F021A
:100568001269D77D02E4FF1269D77D32E4FF126970
:10057800D77D607F021269D77D027F0712519B5099
:10058800057F04127209900528E0F536A3E0F537D7
:100598007F03127209E55A7006A22492298009E5A0
:1005A8005AB40104A2259229E53745367005D22AA6
:1005B800020A1D3029DFE55A7006A2249229800913
:1005C800E55AB40104A22592292029EAE55A700BBC
:1005D800755B1E755C6085455D800EE55AB4010942
:1005E800755B1E755CB085465DE55DD39400500370
:1005F800020A17855C82855B83E0640B6003020A4C
:1006080012A3E0FFB40A0AE55DB40205D22A020A81
:1006180017EF6401701E120D33A3E0640A7015E52C
:100628005D6405700F120D33120D73120A481233F0
:10063800CE020A17120D33E0B40111120D33A3E0F4
:10064800B40109120EF21219BB020A17120D33E097
:100658006401701E120D33A3E064027015E55D6439
:1006680005700F120D33120D73120A4812649B02A3
:100678000A17120D33E06401701D120D33A3E064F4
:10068800037014E55DB4050F120D33120D73FDAB45
:100698005A123C2E020A17120D33E0B4011D120D36
:1006A80033A3E0B40415E55DD39405400EAB5AAD11
:1006B8005CAC5BAF5D12329A020A17120D33E0642C
:1006C80001701D120D33A3E064057014E55DB405D7
:1006D8000F120D33120D73FDAB5A125DB9020A17D2
:1006E800120D33E06401701D120D33A3E06406702F
:1006F80014E55DB4050F120D33120D73FDAB5A12DC
:100708005083020A17120D33E0B4011D120D33A3F2
:10071800E0B40715E55DD39405400EAB5AAD5CAC6B
:100728005BAF5D1249C0020A17120D33E064017015
:100738001D120D33A3E064087014E55DB4050F12B3
:100748000D33120D73FDAB5A1264D5020A17120D40
:1007580033E0B40215120D33A3E0B40A0DE55DB41D
:100768000308AF5A126694020A17120D33E0B40256
:1007780016120D33A3E0B4010EE55DB40E09120E96
:10078800F4123024020A17120D33E0B40216120DC7
:1007980033A3E0B4020EE55DB40709120EF4125655
:1007A80022020A17120D33E0B40215120D33A3E02A
:1007B800B4090DE55DB40308AF5A125857020A1779
:1007C800120D33E064027019120D33A3E0B409115D
:1007D800E55DB4040C120D33120F69126A7D020A2A
:1007E80017120D33E064037021120D33A3E0640A7D
:1007F8007018E55D64057012120D33120D73FD1249
:1008080070B5AD5A124A75020A17120D33E0640327
:100818007029120D33A3E064017020E55DD39405BF
:100828004019120D33120D73FD1270B5855A62AB63
:100838005DAD5CAC5B1240A0020A17120D33E06498
:10084800037021120D33A3E064027018E55D64059E
:100858007012120D33120D73FD1270B5AD5A12627B
:10086800F4020A17120D33E0B40315120D33A3E096
:10087800B4030DE55DB40308AF5A126370020A179A
:10088800120D33E0B40318120D33A3E0B40410E5DD
:100898005DD394034009120F52124D14020A171225
:1008A8000D33E0B40315120D33A3E0B4050DE55D77
:1008B800B40308AF5A1270A3020A17120D33E0B43A
:1008C8000316120D33A3E0B4060EE55DB405091254
:1008D8000EF4126BB7020A17120D33E06403701995
:1008E800120D33A3E0B40711E55DB4040C120D3307
:1008F800120F69126EC1020A17120D33E0B4031603
:10090800120D33A3E0B4080EE55DB40409120EF429
:10091800126BDC020A17120D33E064057014E55DF2
:10092800B4040F120D29A3A3E0FDAB5A1222110241
:100938000A17120D33E0B40516120D77B40B10E543
:100948005DD394054009120F52123627020A171276
:100958000D33E064067014E55DB4040F120D29A38D
:10096800A3E0FDAB5A122403020A17120D33E0B4B8
:100978000616120D77B40B10E55DD39405400912E5
:100988000F5212293E020A17120D33E06409701A39
:10099800120D33A3E0B40A12E55DB4040D120D3351
:1009A800A3A3E0FF126056020A17120D33E0640990
:1009B8007018120D33A3E0B40110E55DB4040B12F6
:1009C8000D33120F691265F08045120D33E0B4093A
:1009D80017120D33A3E0B4020FE55DD39404400869
:1009E800120EF212176D8027120D33E06409701A87
:1009F800120D33A3E0B40310E55DB4040B120D33FC
:100A0800120F69125FC480078000AF5A126EDE2091
:100A18002A0302059DC21ED22DAF5A125CC77D6003
:100A28007F021269D77D327F031269D77F03127262
:0F0A3800091260E57FFF1271C8E47884F6C223CB
:080A470022FD1270B5AD5A2228
:0819BB008E5E8F5F8D608B6171
:1019C300120EE0FFE55F2404120D88FD1267D28F2B
:1019D3006274E22562F562C394005003021BBCE506
:1019E3006294144003021BBCE5616406701D120D72
:1019F30084B4010C120DCC120E997401F0021BB8C1
:101A0300120DCC120E99E4F0021BB8E561640E606E
:101A130003021ADAE55F240C120D88FFB40A14E5F9
:101A23005F240D120D88B40A0A120DCC120E29E49C
:101A3300F08013E55F240D120D88FD126F35120D32
:101A4300CC120E29EFF0E55F240A120D88FFB40AC9
:101A530014E55F240B120D88B40A0A120DCC120E82
:101A630077E4F08013E55F240B120D88FD126F35C8
:101A7300120DCC120E77EFF0E55F2409120D88FFEB
:101A8300640A6006EFD39409400A120DCC120E4D7E
:101A9300E4F08010E55F2409120D88FF120DCC12CB
:101AA3000E4DEFF0120D84FFB40B15E55F24061203
:101AB3000D88B40B0B120DCC120E0374FFF08008CB
:101AC300121BE8120E03EFF0121BC4120DC1120E0B
:101AD300997401F0021BB8E561640A706E120DCCB3
:101AE300120E29E4120DCB120E77E4F0E55F240900
:101AF300120D88FF640A6006EFD39409400A120DA1
:101B0300CC120E4DE4F08010E55F2409120D88FF1E
:101B1300120DCC120E4DEFF0120D84FFB40B15E530
:101B23005F2406120D88B40B0B120DCC120E037436
:101B3300FFF08008121BE8120E03EFF0121BC41211
:101B43000DC1120E997401F0021BB8E561640970AE
:101B530068120DCC120E29E4120DCB120E77E4128B
:101B63000DCB120E4DE4F0120D84FFB40B15E55F9F
:101B73002406120D88B40B0B120DCC120E0374FF46
:101B8300F08013E55F2406120D88FD126F35120DE8
:101B9300CC120E03EFF0E55F2407120D88FFE55F1B
:101BA3002408120D88FD126F35120DCC120DC112CF
:101BB3000E997401F0D22C8002C22CAF6012719E78
:101BC30022E55F2407F582E4355EF583E0FFE55FF8
:101BD3002408F582E4355EF583E0FD126F35E56296
:101BE30075F007A422E55F2406F582E4355EF583EC
:0C1BF300E0FD126F35E56275F007A422DA
:1033CE008F5E8D5FE55ED3941D50030234DAE55EA9
:1033DE00943240030234DAD22DAF5F125CC77D46C1
:1033EE007F071269D7AF5E12384E74E2255EF55E26
:1033FE00120E25E07021120E71E0701B120E47E0C6
:10340E007015120DFDE0700F120F41700A1234F399
:10341E007D537F020234D01234E2E55E75F007A4CC
:10342E00120E99E070047D3680027D387F06126997
:10343E00D71234E2120E23E0FFD394014034EF94FE
:10344E0013502F7D097F061269D7120E231234EA0C
:10345E007FF47E01126F6D7D0E7F031269D77D356D
:10346E007F061269D77D097F061269D7120E711277
:10347E0034EA7FF47E01126F6D120E47E0FF600595
:10348E00125D6A800A1234F37D0F7F031269D77DB5
:10349E00277F021269D7120DFDE0FFF46008126F4C
:1034AE00F212384E80077D187F021269D77D377F62
:1034BE00041269D7120F41FF126FF212384E7D05BA
:1034CE007F061269D7C22DAF5F025CC7C22CAF5FF9
:1034DE0012719E227FF47E01126F6D22E0FF126F39
:0D34EE00F212384E227D187F021269D7229B
:02649B008D5E14
:10649D00EFD3941D402AEF9432502574E22FFFE480
:1064AD00FEEEFD3395E0FCEF75F007A42450F58268
:1064BD00E4340A120E3AE4F00EBE07E5D22C800247
:0764CD00C22CAF5E12719EAC
:0164D40022A5
:063024008E5E8F5F8D60DF
:10302A00D22B120EE0FFE55F2404120DA212314BDF
:10303A00C39418501C855F82855E83A3A3A3E0FF17
:10304A00E55F2404120DA2FD12707D7882A6078026
:10305A0006E47882F6C22B120D9112314BC3943CCE
:10306A00500D120D91FD12707D7883A6078006E43B
:10307A007883F6C22BE55F2407120DA2FF12713086
:10308A008F61E561D394004017E56194085011E51A
:10309A005F2407120DA2FF127130787FA6078006FF
:1030AA00787F7601C22BE55F2408120DA2FFE55F47
:1030BA002409120DA2123154401FE56194205019BF
:1030CA00E55F2408120DA2FFE55F2409120DA2FD97
:1030DA0012707D7887A607800678877601C22BE56D
:1030EA005F240A120DA2FFE55F240B120DA2123112
:1030FA0054401FE561940D5019E55F240A120DA290
:10310A00FFE55F240B120DA2FD12707D7880A607E1
:10311A00800678807601C22BE55F240C120DA2FF8F
:10312A00E55F240D120DA2FD12707D7881A607308D
:10313A002B07125BBED22C8002C22CAF6012719E8A
:10314A0022FD1267D28F61E56122FD1267D28F617B
:06315A00E561D3940022A0
:065622008E5E8F5F8D60BB
:10562800D22B120EE0FFE55F2404120E6812568D8D
:105638009418501C855F82855E83A3A3A3E0FFE5D1
:105648005F2404120E68FD12707D7882A60780061A
:10565800E47882F6C22B120E5712568D943C500DE8
:10566800120E57FD12707D7883A6078006E47883B2
:10567800F6C22B302B07125BBED22C8002C22CAF95
:045688006012719E9D
:0B568C0022FD1267D28F61E561C3228E
:10713000120EC04008EF6480948A5001227F002222
:10707D00AE05127130EFC454F0FDAF06127130EF52
:03708D004DFF2292
:106694008F5ED22D125CC77D1E7F081269D77D26BE
:1066A4007F081269D77D527F041269D7C22B126BFF
:1066B40091125F30787FE6FF125D6A125C71C22D21
:0666C400AF5E125CC7226C
:106A7D008D5EEFD3940A4006EFD3940F4003EF7071
:106A8D000E90002BEFF0D22CAF5E12719ED322C26E
:086A9D002CAF5E12719EC322B2
:025857008F5E62
:10585900D22D125CC77D207F051269D77D2E7F036B
:105869001269D77D527F041269D790002BE0F55F4A
:10587900E55FB40B067D5F7F078034E55FB40C06F6
:105889007D5E7F068029E55FB40D067D0A7F028073
:105899001EE55FB40E067D327F028013E55FB40F0B
:1058A900067D467F028008E55F70077D0A7F031247
:0958B90069D7C22DAF5E125CC775
:0158C20022C3
:106EC1008D5E120EC0400EEF6480948650071267EB
:0D6ED1006AD22C8002C22CAF5E12719E228C
:026BB7008D5EF1
:106BB900120EC71267D2120EC04010EF648094A162
:106BC9005009900029EFF0D22C8002C22CAF5E123E
:026BD900719EAB
:016BDB002297
:026BDC008D5ECC
:106BDE00120EC71267D2120EC04010EF648094A13D
:106BEE005009900028EFF0D22C8002C22CAF5E121A
:026BFE00719E86
:016C00002271
:10709000D3EF648094814008EF6480948A50012289
:0370A0007F00224C
:10714000120EC04008EF648094A15001227F0022FB
:08176D008E5E8F5F8D608B61C1
:10177500120EE014F56374FC2561F5616403600FD6
:10178500E56164076009E561640B6003021958C3EC
:10179500E563648094805003021958E5636480947E
:1017A500884003021958E4F562120D6A7803C333C1
:1017B500CE33CED8F92430F58274003EF583AF627E
:1017C500EF3395E0FE120DE5E4F00562E562B4083D
:1017D500D8756204E56164037029120D4612199EDD
:1017E500120D687803C333CE33CED8F9120D3BA35F
:1017F500A3120D637803C333CE33CED8F9120FCAC3
:1018050002194FE56164077069120D4612199E129F
:101815000D687803C333CE33CED8F9120D3BA3A39D
:10182500120D637803C333CE33CED8F9120FCA1223
:101835000D41A3A3A3120D637803C333CE33CED8D2
:10184500F92432F5827400120D41121960C333CEAA
:1018550033CED8F92433F5827400120D41120D5898
:101865007803C333CE33CED8F92434F5827400021D
:10187500194FE561640B6003021958120D46E01219
:101885000EFBA3E0FD1267D2127140120D687803BA
:10189500C333CE33CED8F9120D3BA3A3120D637813
:1018A50003C333CE33CED8F9120FCA120D41A3A309
:1018B500A3120D637803C333CE33CED8F92432F5A2
:1018C500827400120D41121960C333CE33CED8F99C
:1018D5002433F5827400120D41120D587803C33379
:1018E500CE33CED8F92434F5827400120D41E58249
:1018F5002407120D5C7803C333CE33CED8F92435D3
:10190500F5827400120D41E5822408120E1A120E9A
:10191500FBE5822409120E1AFD1267D212714012DC
:101925000D687803C333CE33CED8F92436F58274E7
:1019350000120D41E582240A120D5C7803C333CEF3
:1019450033CED8F92437F58274003EF583EDF0D215
:0A1955002C8002C22CAF6012719EBC
:10195F0022E5822404F582E43583F583E0FFE56216
:10196F00FD3395E0FCE55F2DF582E55E3CF583E503
:10197F00822405F582E43583F583E0FD1267D212E8
:10198F007140AD07AF63EF3395E0FEEF780322E0D0
:10199F00FFE562FD3395E0FCE55F2DF582E55E3CEA
:0C19AF00F583A3E0FD1267D21271402204
:045FC4008D5EAC073B
:105FC800D3EC648094804035EC64809489502EE44E
:105FD800FDECFF3395E0FEEF7803C333CE33CED824
:105FE800F92428F58274003EF583EDFF3395E0FE31
:105FF800120DE5E4F00DBD08D8D22C8002C22CAFFA
:046008005E12719E15
:01600C002271
:1065F0008D5E120EC0402FEF648094895028EF14F6
:10660000FFE55E24FF922B1252AAD22DAF5E125CE0
:10661000C77542017F327E00126F6DE54270FCC289
:076620002DAF5E125CC722E2
:0849C0008F5E8C5F8D608B613E
:1049C800856082855F83120E0DFD1267D28F62E5C6
:1049D80062D394005003024A6DE5629433400302A7
:1049E8004A6DE55E64067036D22DAF61125CC77DF4
:1049F800527F051269D7AF6212384E120F29B401DF
:104A08000A120E817401F07D388007120E81E4F0DD
:104A18007D367F061269D7C22DAF61025CC7E5609B
:104A28002406120F2D640B703C120F29B4010812D2
:104A38000E817401F08005120E81E4F074F9255E90
:104A4800F55E75F0041211A5AFF0EF7014E560245F
:104A580006FBE4355FFAAD62E4FF12374ED22C80D4
:0C4A680006C22C8002C22CAF6112719EAD
:014A7400221F
:08329A008F5E8C5F8D608B617B
:1032A200856082855F83120E0DFD1267D28F62E503
:1032B20062D3940050030233C6E5629429400302AC
:1032C20033C6E55E64067037D22DAF61125CC77DEE
:1032D200527F051269D7AF6212384E120EB4E0B4B3
:1032E200010A120E8D7401F07D388007120E8DE4F2
:1032F200F07D367F061269D7C22DAF61025CC7E549
:10330200602406120EB8E0640B60030233C6120E8C
:10331200B4E0B40108120E8D7401F08005120E8D16
:10332200E4F0E4FFFEE5602407120EB8E5822E12F7
:103332000E1AB40B04AF0680040EBE08E8EF700349
:103342000233C6C39408507C120F36EFF07E01EFB1
:103352002401FDE433FCEEC39DEC6480F874809894
:103362005020E5602406120EB8E5822E120E1AFDD8
:10337200120F36E5822EF582E43583F583EDF00EE9
:1033820080CDE5602408120EB8E5822F120E1A6471
:103392000B602DEF2408FEC3E55E9EF55E75F0041A
:1033A2001211A5AEF0EE701CE5602407FDE4355F56
:1033B200FC7E00ED2FFBEE3CFAAD627F0112374E30
:0B33C200D22C8002C22CAF6112719E61
:0133CD0022DD
:08374E008F638D648A658B66B0
:10375600756801E4F567120DAFE0FF6409703E126B
:10376600383F8003120F0ED8FB120DAB123831789A
:1037760008EF088003120F0ED8FB120DABA3A3E0CF
:10378600FFE568FD3395E0FCE5662DF582E5653CD1
:10379600F583A3A3A3E0FD1270B50237EA120DAFBD
:1037A600E0FF12383F8003120F0ED8FB120DAB124A
:1037B60038317804EF088003120F0ED8FB120DABD8
:1037C600A3A3E0FF1271FFEF426AAE69AF6A780405
:1037D600EF088003120F0ED8FB120DABA3A3A3E0D4
:1037E600FF1271FFEF426AE563700FAF67120D6C4F
:1037F600120EAAE564900AC08012E563B40117AF01
:1038060067120D6C120EAAE564900530120DE2E502
:1038160069F0A3E56AF074042568F5680567C3E5F1
:0A3826006764809490500302375C41
:1038300022A3E0FF1271FFEF426AAE69AF6A221263
:0E38400071FF7569008F6AAE697804EF082287
:0A71FF00EFD3940940037F00222221
:023C2E008B5EAB
:103C30001267D28F61E561D394005003023D10E515
:103C40006194334003023D10D22DAF5E125CC77DFC
:103C5000527F051269D7AF6112384E746F25611219
:103C60000E91E060047D3880027D367F061269D7B0
:103C70007F2C7E01126F6DE561120F38E0F55F70E9
:103C8000077D1B7F061269D77D577F021269D7E532
:103C90005F603B756001AF5F120D6C2401FFE43E75
:103CA000FEAD60ED3395E0FCC3ED9FEE6480F8EC73
:103CB0006480985019120DD3E0B40A04E4FD800624
:103CC000120DD3E0FDE4FF1269D7056080C87F2C98
:103CD0007E01126F6DE561900530120F8490000037
:103CE000EEF0A3EFF04E70077D1B7F061269D77DC3
:103CF0000C7F031269D7900000E07002A3E0600916
:103D0000E56114FD7F01122D86C22DAF5E025CC7F6
:073D1000C22CAF5E12719E90
:013D17002289
:025083008B5E42
:105085001267D28F5FE55FD394004077E55F943375
:105095005071D22DAF5E125CC77D527F051269D764
:1050A500AF5F12384E749F255F120E85E060047D58
:1050B5003880027D367F061269D77F2C7E01126FFC
:1050C5006D7F2C7E01126F6DE55F900AC0120F8413
:1050D500900000EEF0A3EFF04E70077D1B7F0612E7
:1050E50069D77D0C7F031269D7900000E07002A399
:1050F500E06009E55F14FDE4FF122D86C22DAF5E69
:0A510500025CC7C22CAF5E12719E5F
:01510F00227D
:0264D5008B5EDC
:1064D7001267D2AD07EDD394004025ED94335020D9
:1064E700E4FC120EA3ED900AC0120DE2E4F0A3F053
:1064F7000CBC10EE749F2D120E85E4F0D22C800296
:07650700C22CAF5E12719E71
:01650E00226A
:025DB9008B5EFF
:105DBB001267D2AD07EDD394004036ED94335031DA
:105DCB00E4FC120EA3ED900530120DE2E4F0A3F00B
:105DDB000CBC10EE746F2D120E91E4F0FCECFF3343
:105DEB0095E0FEED120DDCE4F00CBC08F0D22C803B
:085DFB0002C22CAF5E12719E82
:015E0300227C
:042D86008F628D6368
:102D8A00E4F564E5627052AF64120D6C25E0FDEE65
:102D9A0033FCAF63120D6C7805C333CE33CED8F94A
:102DAA00120E33120F908003120F15D8FB120F70F8
:102DBA008003120F15D8FB540FF566AF63120D6C22
:102DCA007805C333CE33CED8F9120E33120F9C8056
:102DDA0003120F15D8FB022E44E56264017064AF3A
:102DEA0064120D6C25E0FDEE33FCAF63120D6C78B6
:102DFA0005C333CE33CED8F92450F5827405120EAA
:102E0A0039120F908003120F15D8FB120F7080032E
:102E1A00120F15D8FB540FF566AF63120D6C7805C7
:102E2A00C333CE33CED8F92450F5827405120E3945
:102E3A00120F9C8003120F15D8FB540FF567ED543F
:102E4A000FF568E565700CE5667008E5677004E5DE
:102E5A0068607CAD65E4FF1269D7AD66E4FF12696C
:102E6A00D7E56564097045856769AF69FE7804EF3F
:102E7A00088003120F0ED8FBF569E5684269E56917
:102E8A00B4990B7D09E4FF1269D77D098027E569AA
:102E9A0075F00A84F56AFDE4FF1269D7E56A75F0F0
:102EAA000AA4FFC3E5699FF56AFD8009AD67E4FFDF
:102EBA001269D7AD68E4FF1269D77FF47E01126FF9
:0F2ECA006D0564C3E564648094A05003022D8DF0
:012ED90022D6
:1067D200EFD394004015EF940B5010EFC3940A507E
:1067E20008EF75F00AA4FE8002E4FEEDD3940040A7
:1067F2000EED940B5009EDC3940A5003ED2EFEAF3B
:01680200068F
:016803002272
:064D14008E5E8F5F8B60D4
:104D1A00756105756240D3ED64809484407CED64CE
:104D2A008094A55075ED24FDF563D39401406BE59D
:104D3A006320E06613F5640562E562AE6170020500
:104D4A006114F5828E83E564F07403255FF55FE4F0
:104D5A00355EF55EE4F563E563C395645033855FBC
:104D6A0082855E83E0FFA3E0FD1270B50562E5620D
:104D7A00AC617002056114F5828C83EFF0055FE582
:104D8A005F7002055E055FE55F7002055E05638080
:104D9A00C6D22CAF6012719ED322C22CAF601271A0
:024DAA009EC3A6
:014DAC0022E4
:0440A0008C5F8D6044
:1040A400120EC05003024178EF64809495400302DD
:1040B4004178EB648094875003024178EB648094E8
:1040C400E44003024178120D6C7805C333CE33CE3D
:1040D400D8F9120FD1F5638F64EB24FBF565D39403
:1040E400025003024178E56575F00384E5F060034E
:1040F400024178E56575F00384F567C39410507444
:10410400120F7D7002056314F5828E83E567F074E7
:1041140005120FDBE4F565E565C395675052120F90
:10412400E5E0F566B40A10120F7D7002056314F51C
:10413400828E83E4F0800F120F7D7002056314F504
:10414400828E83E566F0120FE5A3E0FF120FE5A36C
:10415400A3E0FD1270B58F66120F7D700205631423
:10416400F5828E83E566F07403120FDB056580A784
:0B417400D22C8002C22CAF6212719EA0
:01417F00221D
:08293E008E5E8F5F8D608B61DE
:10294600C22B120FEC60030229DB122AB6500302D7
:1029560029D6E5649408E56394075074C3E560647A
:1029660080948A506B120EE9A3E0F562B4010690DA
:102976000520022A2BE562B40206900522022A2BC4
:10298600E562B40306900524022A2BE562B4040628
:10299600900526022A2BE562B40506900528022A30
:1029A6002BE562B4060690052A022A2BE562B407D7
:1029B6000690052C022A2BE562B4080590052E80A8
:1029C60064E562B40905900530805AD22B022AA725
:1029D600D22B022AA7120EE9E064017052AD60AF55
:1029E6005FAE5E122AB65003022AA7E5649408E594
:1029F6006394074003022AA7C3E5606480948A4073
:102A060003022AA7120EE9A3E0F562B40A059005AF
:102A1600328012E562B401059005348008E562B49F
:102A26000209900536E563F0A3806FD22B807212FF
:102A36000EE9E06402706AAD60AF5FAE5E125E04DE
:102A46007563008F64C3E5649463E5639400505135
:102A5600C3E560648094885048120EE9A3E0F562ED
:102A6600B40107900538EFF08037E562B4020590AF
:102A760005398026E562B4030590053A801CE562B7
:102A8600B4040590053B8012E562B4050590053C4B
:102A96008008E562B4060890053DE564F08002D240
:0F2AA6002B302B04C22C8002D22CAF6112719EF8
:102AB50022124C708E638F64D3E564943BE5639476
:022AC5000022ED
:064C70008E658F66A905A8
:104C76007D057C00120FB4E0C3940A4005120FB400
:104C8600E4F00DBD00010CED640A4C70E7B90607AF
:104C9600120DF0FF7E0022E964077010120DF07508
:104CA600F00AA4ACF0FDE5662406801BE9640870F2
:104CB60021120DF075F064A4ACF0FDE56624061231
:104CC6000DF4120F1C2407120DF42DFDE43CAF0564
:104CD600FE22E964097033120DF0FF7E007C037D2D
:104CE600E81211C7AC06AD07E5662406120DF47589
:104CF600F064120F1F2407120DF4120F1C24081261
:0D4D06000DF42DFDE43CFEAF0522E4FEFFA0
:014D1300227D
:065E04008E658F66A90502
:105E0A007F057E00120FBFE0C3940A4005120FBF40
:105E1A00E4F00FBF00010EEF64084E70E7E9640773
:105E2A007020E5662405F582E43565F583E075F0B2
:105E3A000AA4FFE5662406F582E43565F583E02FBA
:045E4A00FF227F00B4
:015E4E002231
:083627008E5E8F5F8D608B61E8
:10362F00C22BD3E5606480948450030236D5E560E5
:10363F006480948D40030236D5120FEC600302367E
:10364F00D5120EE012126B367501368002368B03DF
:10365F00369504369F0536A90636B30736BD0836AC
:10366F00C709000036D1756201756300D22B02378E
:10367F000C756201756308D22B02370C75620175E8
:10368F006310D22B8077756201756318D22B806D12
:10369F00756201756320D22B806375620175632893
:1036AF00D22B8059756201756330D22B804F7562B2
:1036BF0001756338D22B8045756201756340D22B3B
:1036CF00803BC22B8037D3E56064809484402EE525
:1036DF00606480948D5026855F82855E83A3A3E00E
:1036EF00B4011A855F82855E83A3A3A3E024F670DD
:1036FF000A756201756358D22B8002C22B302B37AB
:10370F00E4FF120F5BE4F00FBF08F7E56024FB85C1
:10371F006382856283F07F01E55F2404F582E435DF
:10372F005EF583E5822F120E1AFE120F5BEEF00F7D
:0E373F00BF08E5D22C8002C22CAF6112719E31
:01374D002259
:044A75008F5E8D5F64
:104A7900E55ED394005003024B18E55E941540039C
:104A8900024B18D22DAF5F125CC77D5F7F0512699B
:104A9900D7AD5EE4FF1269D77D527F041269D77FD3
:104AA900F47E01126F6D75F020E55E90028012129E
:104AB9005FAF828583628F63E0F560603DD39400C8
:104AC9004046E56094105040E56025E0F560756169
:104AD90001E5602401FFE433FEC3E5619FEE6480D4
:104AE900F87480985022120FA8E0FF120FA8A3E0D3
:104AF900FD1268640561056180D77D1B7F06126917
:104B0900D77D5F7F051269D7C22DAF5F025CC7C22F
:064B19002CAF5F12719E3B
:014B1F002273
:102403008F5E8D5F8B60E55E640A7074E55FC394D5
:102413000A40030225701225A6E4FDFF1269D7AD19
:102423005F12257FE55F12126B244B0124510224B6
:102433005703245D04246305246906246F07247568
:1024430008247B09000024809005200224CA9005FB
:10245300220224CA9005240224CA9005260224CA13
:102463009005280224CA90052A0224CA90052C024A
:1024730024CA90052E0224CA900530804A02256999
:10248300E55E64017052E55FD394004006E55F9416
:10249300034006E55F640A703C1225A6E55FB40AB3
:1024A3000A7D0A12257F900532801CE55FB4010A7C
:1024B3007D0B12258C900534800DE55FB402137DEE
:1024C3000C12258C900536E0FEA3E0FF126735025F
:1024D3002577022569022570E55E64026003022503
:1024E30077E55FD394005003022570E55F940750AE
:1024F3007CD22DAF60125CC77D277F081269D77D20
:1025030006E4FF1269D77D14E4FF1269D7E55F245F
:10251300FE601A14602114602814602F146036249E
:102523000570437D0112259990053880307D021294
:10253300259990053980267D031225BC90053A80A4
:102543001C7D041225BC90053B80127D051225C914
:1025530090053C80087D061225C990053DE0FF7E6D
:1025630000126804800EAF60126EDE8007C22CAFCB
:102573006012719EC22DAF60125CC722E4FF126924
:10258300D77D527F041269D722E4FF1269D77D52A7
:102593007F041269D722E4FF1269D77D527F0412A8
:1025A30069D722D22DAF60125CC77D277F081269DD
:1025B300D77D06E4FF1269D722E4FF1269D77D5263
:1025C3007F041269D722E4FF1269D77D527F041278
:0325D30069D722A3
:044E43008E638F6487
:104E47000564E5647002056314F5828E83E0F566F8
:104E5700607AC3940850757F2C7E01126F6DE4F55C
:104E670065E565C395665064856482856383E01252
:104E7700126B4EB4004E920A4E960B4E9C0C4EA2ED
:104E87000D4EA80E4EAE0F00004EBAE4FD802D7DEC
:104E97005F7F0780287D5E7F0680227D0A7F0280F4
:104EA7001C7D327F0280167D467F0280107D0A7F3F
:104EB70003800A856482856383E0FDE4FF1269D776
:0C4EC7000564E5647002056305658095D4
:014ED30022BC
:062211008F5E8D5F8B6003
:10221700C22BE55E640A6003022305E55F12126BB9
:10222700224601225902226C03227F0422920522B0
:10223700A80622BE0722D40822E9090000230112BA
:10224700233A7D01122388756101756200D22B0242
:10225700232112233A7D02122388756101756208D2
:10226700D22B0223211223567D0312239575610178
:10227700756210D22B0223211223567D0412239557
:10228700756101756218D22B022321122372122362
:10229700E87D051223B8756101756220D22B0223F0
:1022A700211223721223E87D061223B87561017586
:1022B7006228D22B0223211223A21223FC7D0712AC
:1022C70023C5756101756230D22B0223211223A227
:1022D7001223FC7D081223C5756101756238D22B64
:1022E70080381223D2E4FDFF1269D77D091223EF4C
:1022F700756101756240D22B8020C22B801CE55E80
:1023070064017016E55F24F670101223D27D0A125D
:1023170023EF756101756258D22B302B09AF62AE7E
:1023270061124E438005AF60126EDEC22DAF6012A0
:022337005CC781
:1023390022D22DAF60125CC77D577F021269D77D0B
:1023490005E4FF1269D7E4FDFF1269D722D22DAF48
:1023590060125CC77D577F021269D77D05E4FF12C1
:1023690069D7E4FDFF1269D722D22DAF60125CC78D
:102379007D577F021269D77D05E4FF1269D722E4F0
:10238900FF1269D77D527F041269D722E4FF1269CF
:10239900D77D527F041269D722D22DAF60125CC754
:1023A9007D577F021269D77D05E4FF1269D722E4C0
:1023B900FF1269D77D527F041269D722E4FF12699F
:1023C900D77D527F041269D722D22DAF60125CC724
:1023D9007D577F021269D77D05E4FF1269D722E490
:1023E900FDFF1269D722E4FF1269D77D527F0412DB
:0A23F90069D722E4FDFF1269D72224
:10384E008F72E572D3945940107D5A12393524A6E1
:10385E00FD700302393402392FE572D3944F4016AE
:10386E00E572945A50107D5012393524B0FD700314
:10387E0002393402392FE572D394454016E572941D
:10388E005050107D4612393D24BAFD700302393472
:10389E0002392FE572D3943B4012E5729446500CD8
:1038AE007D3C12393D24C4FD607C8075E572D39455
:1038BE00314012E572943C500C7D3212394524CEC3
:1038CE00FD6063805CE572D394274012E5729432FA
:1038DE00500C7D2812394524D8FD604A8043E5728C
:1038EE00D3941D4016E572942850107D1EE4FF12ED
:1038FE0069D7E57224E2FD602D8026E572D394131C
:10390E004016E572941E50107D14E4FF1269D7E53F
:10391E007224ECFD60108009E572C394145007AD5B
:10392E0072E4FF1269D722E4FF1269D7E57222E42E
:0F393E00FF1269D7E57222E4FF1269D7E5722202
:105CC7008F6AE56A700C302D097F0112721C7FC044
:105CD700801FE56A700C202D097F011272097FC0B1
:105CE7008026E56AB40112302D0F7F0212721C7FE5
:105CF70030120016C22F026C93E56AB40114202DEE
:105D0700117F021272097F301271C87FC87E00129C
:035D17006F6D228B
:106C6F008F69D22D125CC77D607F021269D77D328A
:106C7F007F061269D77D1E7F051269D7C22DAF69B6
:046C8F00125CC722AA
:106EDE008F69D22D125CC77D607F021269D77D301B
:0D6EEE007F031269D7C22DAF69125CC72265
:0E719E008F68302C03026C6FAF68126EDE2219
:10605600EF24FE60101460162402701C7F01127279
:106066001C7F8080107F0212721C7F2080077F03B6
:1060760012721C7FA01200167FF47E01126F6D75DE
:106086004204E54270FC7F647E00126F6D7F03124E
:0860960072097FA01271C822FB
:106804008E618F627C007D0A1211D9AD07E4FF12FC
:1068140069D77D5B7F061269D7AE61AF627C007D6C
:106824000A1211D9E4FF1269D77D4A7F070269D79A
:046735008E618F6280
:106739007C007D3C1211D9AA06AB0712384E7D05A3
:106749007F061269D7AE61AF627C007D3C1211D918
:10675900ED4C600CAF0512384E7D4A7F071269D7A0
:01676900220D
:0262F4008D5EBD
:1062F600120EC0402FEF648094955028120D6C78D2
:1063060005C333CE33CED8F9120FD1FEE4FD0FEF1D
:10631600AA0670010E14F5828A83E4F00DBD20EE04
:0B632600D22C8002C22CAF5E12719ED0
:016331002249
:106370008F5E900540E0C394014015D22D125CC79A
:106380007542037F327E00126F6DE54270FC80150E
:10639000D22DAF5E125CC77D1B7F061269D77D0CC4
:0D63A0007F031269D7C22DAF5E125CC722C9
:1070A3007E10900540E4F0A3DEFC7E10D22C12711A
:0170B3009E3E
:0170B40022B9
:1070B500BF0A02E4FFBD0A02E4FDEF75F00AA42D44
:0270C500FF22A8
:106F3500EFD394094002E4FFEDD394094002E4FD48
:0C6F45007804EF08800123D8FD4DFF22E6
:104325000701020304050607070706050403020142
:1043350003010A0A030307050303020503020A0A28
:1043450004050A0A0104050A0A0A04050A0A020301
:10435500070A0A03040A0A04024B00020032072E68
:1043650003024B0002003202055F000302055F00F5
:104375000402055F000502055F000604072E0826F6
:104385000640033204072E08260640025304081E81
:1043950008260452010008024B00020032072E08CD
:1043A5001E08260452010003072B023506360307B3
:1043B5002B0235063803072B0235072603072B0288
:1043C50035025302055F000F02055F001002055F0D
:1043D500001102055F001202055F001302055F0070
:0A43E50014080C0A1D020500241B39
:1055A9007461F0A37420F0A37452F0A37401F0A302
:1055B90022A3F0A37461F0A37440F022F0A3740352
:1055C900F0E4A3F0A37410F0A37403F0E4A3F0A330
:1055D900227461F0A37441F0A3227461F0A3F0A3D3
:1055E9007430F0A3227496F0A37432F0A37495F08A
:1055F900A3741EF0A322F0A37461F0A314F0A374A2
:1056090070F0A3E4F022A3F0A37452F0A3223CF5B6
:0956190083E0FEEF3395E0FC2272
:10003E007E437F257C017D507B081261F27E437FDB
:10004E002D7C017D587B081261F27E437F357C0149
:10005E007D007B041261F27E437F417C017D087B33
:10006E00041261F27E437F3D7C017D107B041261A0
:10007E00F27E437F397C017D187B041261F27E4350
:10008E007F4A7C017D207B051261F27E437F457C99
:10009E00017D287B051261F27E437F4F7C017D300E
:1000AE007B051261F27E437F547C017D387B041206
:1000BE0061F27E437F587C017D407B041261F27EAB
:1000CE00437F5C7C027DA07B091261F27E437F65DB
:1000DE007C027DC07B071261F27E437F6C7C027DC9
:1000EE00E07B051261F27E437F717C037D007B0510
:1000FE001261F27E437F767C037D207B051261F2D6
:10010E007E437F7B7C037D407B051261F27E437FC5
:10011E00807C037D607B091261F27E437F897C03C4
:10012E007D807B091261F27E437F927C037DA07BF2
:10013E00091261F27E437F9B7C037DC07B111261AD
:10014E00F27E437FAC7C037DE07B071261F27E433F
:10015E007FB37C047D007B071261F27E437FBA7C05
:10016E00047D207B071261F27E437FC17C047D40BB
:10017E007B071261F27E437FC87C047D607B051293
:10018E0061F27E437FCD7C047D807B051261F27E21
:10019E00437FD27C047DA07B051261F27E437FD724
:1001AE007C047DC07B051261F27E437FDC7C047D86
:1001BE00E07B051261F27E437FE17C057D007B05CD
:1001CE001261F27E437FE67C057D407B091261F26F
:1001DE009000297417F07F0312676A900028741933
:1001EE00F090002074B1F09000217491F0900022F4
:1001FE007403F0900023747FF090002404F09000BC
:10020E00257403F0E4900026F0900027F090003063
:10021E0074091255C57415F0A37403F0A374151266
:10022E0055C57409F0A37403F0E4FFEFFD3395E0B8
:10023E00FC74302DF582740012561774102DF58251
:10024E0074003CF583EEF00FBF08E0E4FFEFFD33E2
:10025E0095E0FC74382DF582740012561774182D23
:10026E00F58274003CF583EEF00FBF08E090052098
:10027E00E4F0A374B4F0900522E4F0A374B4F0900B
:10028E0005247401F0A374E0F0900526E4F0A37445
:10029E0078F09005287402F0A37458F090052AE4C3
:1002AE00F0A3743CF090052C7402F0A37458F07413
:1002BE000790052EF0A3F0900530F0A3F0900532D4
:1002CE00F0A3F0900534F0A3F0900536E4F0A3749B
:1002DE003CF0900538740AF09005397428F09005BA
:1002EE003A7405F090053B740AF090053CF09005C9
:1002FE003D7428F09000A47401F0900B607415F01A
:10030E00A37411F09000A57401F0900B807415F099
:10031E00A37410F09000A67401F0900BA07415F069
:10032E00A37421F09000A77401F0900BC07415F027
:10033E00A37420F09000A87401F0900BE07415F0F7
:10034E00A37431F09000A97401F0900C007415F0B4
:10035E00A37430F09000AA7401F0900C207415F084
:10036E00A37441F09000AB7401F0900C407415F042
:10037E00A37440F09000AC7401F0900C60745312B2
:10038E0055B37438F0A3E4F0A37453F0A3E4F090E3
:10039E0000AD04F0900C8074531255B37434F0A376
:1003AE007421F0A37453F0A3E4F09000AF04F09026
:1003BE000CC01255B17430F0740312560FE4F09065
:1003CE0000B004F0900CE01255B17430F0740412C9
:1003DE00560FE4F09000B104F0900D001255A97480
:1003EE00321255B37452F0A37420F09000B274011F
:1003FE00F0900D201255A97432F0A374021256100B
:10040E007420F09000B37401F0900D4074531255A7
:10041E00B37433F0A3E4F09000B404F0900D6012C6
:10042E0055DA7430F074021255BA9000B57401F0BA
:10043E00900D801255DA7430F074051255BA900092
:10044E00B67401F0900DA01255DA7430F0A3740654
:10045E001255BB9000B77401F0900DC01255DA1210
:10046E0055EE7498F0A3744B1255BB9000B87401FE
:10047E00F0900DE01255DA1255EE7493F0A3741845
:10048E001255BB9000B97401F0900E001255DA743B
:10049E0030F0A374131255BBA37470F0A37402F062
:1004AE009000BA14F0900E201255E37412F0A3745B
:1004BE00701255B37461F0A314F09000BB7401F088
:1004CE00900E401255E374111255FF9000BC04F0CB
:1004DE007461900E601255E574141255FF9000D1A0
:1004EE0004F09011001255DA7492F0A3744BF0A33D
:1004FE007490F0A37402F0A37490F0A37432F074AD
:10050E0099A3F0A3F0A374601255B374911255B36E
:10051E007491F0A3E41255BB90000F7401F01260B9
:10052E00E57F0112721C7F401200167D2F7F07128D
:10053E0069D77D0C7F031269D77D327F061269D78A
:07054E007D1E7F051269D735
:010555002283
:0A61F2008E5A8F5B8C5C8D5D8B5E16
:1061FC00E4F9C3E55E6480F8E96480985028E9FF0F
:10620C003395E0FEE55B2FF582E55A3EF583E4938A
:10621C00FFE9FD3395E0FCE55D2DF582E55C3CF591
:06622C0083EFF00980CCB5
:016232002249
:10592900AF6AEF3395E0FEE56975F008A42428F520
:1059390082E43400F583E5822FF582E5833EF58321
:10594900E0FFE56AFD3395E0FC22AB66AD65AF6427
:10595900223EF583E0FD74B82FF582741D3EF58370
:10596900EDF0056AE56A22EF3395E0FEEF25E0FFE9
:10597900EE33FE22A2E0CE13CE13223CF583EFF0E4
:05598900056AE56A2239
:045E4F008C5B8D5C7F
:105E5300EF6043D201D202D20CE4F55D855C82850A
:105E63005B83E0FEA3E04E6027AF5D125970E55CF3
:105E73002FF582E55B3EF583E0FEA3E0FF1246E8E3
:105E8300922920290B055DC3E55D6480949040CC85
:065E9300C201C202C20CB4
:015E990022E6
:045E9A008C608D612A
:105E9E00EF6043D201D202D20CE4F56285618285B5
:105EAE006083E0FEA3E04E6027AF62125970E56199
:105EBE002FF582E5603EF583E0FEA3E0FF1246E893
:105ECE00922D202D0B0562C3E5626480949040CC28
:065EDE00C201C202C20C69
:015EE400229B
:0446E800AD07AC0668
:1046EC00C22E780CEF08800312597DD8FB540FF5BD
:1046FC00637808AF05AE04EF08800312597DD8FB30
:10470C00540FF5647804AF05AE04EF08800312591A
:10471C007DD8FB540FF565ED540FF566E5636071BC
:10472C00B40108125953123EDE8066E563B40208E8
:10473C00125953126E498059E563B4030812595348
:10474C00123B40804CE563B40408125953126DEAD5
:10475C00803FE563B405081259531227908032E567
:10476C0063B406081259531214FF8025E563B4078D
:10477C00081259531254338018E563B408081259BF
:10478C0053125B63800BE563B40906125953126C28
:03479C0001A22E49
:01479F0022F7
:103EDE008F678D688B69E567B40113900020E0FF52
:103EEE00125C19900020EFF0FD7F20023F9BE567EA
:103EFE00B40211900021123FA1900021EFF0FD7F3E
:103F0E0021023F9BE567B40311900022123FA1905E
:103F1E000022EFF0FD7F22023F9BE567B404109074
:103F2E000023123FAB900023EFF0FD7F23805EE570
:103F3E0067B40516900024123FAB900024EFF0FDFD
:103F4E007F247E001266CA026834E567B4061090BC
:103F5E000025123FB5900025EFF0FD7F25802EE560
:103F6E0067B40710900026123FB5900026EFF0FDC3
:103F7E007F268019E567B40819900027E0FFAB692A
:103F8E00AD68125C19900027EFF0FD7F277E0012BE
:103F9E0066CA22E0FFAB69AD68125C1922E0FFAB86
:103FAE0069AD68125C1922E0FFAB69AD68125C194D
:013FBE0022E0
:105C1900D22FAC07BD01047E018033BD02047E0290
:105C2900802CBD03047E048025BD04047E08801EEB
:105C3900BD05047E108017BD06047E208010BD07B7
:105C4900047E408009BD08047E808002C22FBB010A
:105C590005EE4204800BEB7006EEF452048002C29A
:075C69002F302F03AF0422CE
:015C70002211
:026E49008B6755
:106E4B00C22FEF7016ED7013E5677003025F30E52C
:0B6E5B0067B40107787FE6FF125D6A54
:016E66002209
:063B40008F678D688B69A0
:103B4600E5677007123C26E4FD801AE567B40107B5
:103B5600123C267D01800EE567B4020CAD69AF68A4
:103B66001271AC7D02024BC9E567B40306124253DB
:103B7600C21E22E567B40415AD69AF681267D28F1D
:103B860043754205E5427003023C2580F7E567640C
:103B9600067017E5687013F56A12592974102DF529
:103BA600827400125984B408F022E567640770171E
:103BB600E5687013F56A12592974182DF582740098
:103BC600125984B408F022E56764087027E5687026
:103BD60023E569701FF56AAF6AEF3395E0FE74104E
:103BE6002FF582740012595AB408EC754201E54269
:103BF600602D80FAE56764097025E5687021E5693E
:103C0600701DF56AAF6AEF3395E0FE74182FF582E2
:0F3C1600740012595AB408EC754201E54270FC73
:093C250022AD69AF681271AC22F6
:106DEA008F67AE03AF05E567D394004012E5679459
:106DFA0007500CAD061271ACAD07AF67126A2B22B1
:102790008F678D688B69E5677018E5687014E56967
:1027A00070057F011271C8E5696401600302293D6B
:1027B0008043E567701CE568B40117E56970057F23
:1027C000041271C8E5696401600302293D7F0402B7
:1027D000293AE5677029E56864027023E5697005A8
:1027E0007F051271C8E5696401600302293D90000C
:1027F0000FE0B403057F0102293A7F0502293AE57B
:1028000067B4011BE5687017E56970057F021271F6
:10281000C8E5696401600302293D7F0202293AE5A7
:1028200067B4011CE568B40117E56970057F0812FB
:1028300071C8E5696401600302293D7F0802293AF5
:10284000E56764017029E56864027023E569700535
:102850007F0A1271C8E5696401600302293D900096
:102860000FE0B403057F0202293A7F0A02293AE504
:1028700067B4021BE5687017E56970057F40127147
:10288000C8E5696401600302293D7F4002293AE5F9
:1028900067B4021CE568B40117E56970057F101282
:1028A00071C8E5696401600302293D7F1002293A7D
:1028B000E56764027024E5686402701EE5697005CE
:1028C0007F501271C8E5696401707290000FE0B426
:1028D00003047F4080647F508060E567B40317E5A0
:1028E000687013E56970057F801271C8E56964013D
:1028F000704B7F808044E567B40318E568B401132A
:10290000E56970057F201271C8E5696401702E7F4A
:10291000208027E56764037024E5686402701EE583
:102920006970057FA01271C8E569B4011090000FAD
:0E293000E0B403047F8080027FA01200162214
:1014FF008F678D688B69E5677017AD69AF6812717B
:10150F00AC8E348F35D3E5359400E534940050F527
:10151F0022E567B4011BE568B40116E5697007C2DF
:10152F00307F01123160E5696401600302176C803E
:10153F0058E5676401702BE56864027025E56970F2
:10154F0007C2307F02123160E56964016003021740
:10155F006C90000FE06403700302176CD2307F02AF
:10156F008031E5676401702EE56864037028E569D2
:10157F007007C2307F03123160E5696401600302B6
:10158F00176C90000FE0B40306D2307F018004D2B5
:10159F00307F03023160E5676401702DE5686404F4
:1015AF007027E569700CC2307F011231607F4012E5
:1015BF0071C8E5696401600302176CD2307F0112B4
:1015CF0031607F40120016807CE5676401703AE558
:1015DF006864057034E569700CC2307F02123160A7
:1015EF007F101271C8E5696401600302176C9000E7
:1015FF000FE06403700302176CD2307F0212316068
:10160F007F10120016D22F803EE5676401703BE514
:10161F006864067035E569700CC2307F0312316063
:10162F007F501271C8E5696401600302176CD230F4
:10163F007F0312316090000FE0B403047F408002FB
:10164F007F50120016C22F026C93E5676402702957
:10165F00E56864017023E56970057F10021753E593
:10166F0069B401057F1002175DE56964026003022A
:10167F00176CD22F7F01021769E56764027029E5A5
:10168F006864027023E56970057F20021753E569CE
:10169F00B401057F2002175DE5696402600302173C
:1016AF006CD22F7F02021769E56764027029E56823
:1016BF0064037023E56970057F40021753E569B431
:1016CF0001057F4002175DE5696402600302176C34
:1016DF00D22F7F03021769E56764027023E5686400
:1016EF0004701DE56970047F808059E569B40104B9
:1016FF007F80805AE56964027063D22F7F04805A1D
:10170F00E56764027023E5686405701DE569700480
:10171F007F048030E569B401047F048031E569649A
:10172F0002703AD22F7F058031E5676402702EE593
:10173F0068640670287D017F0712519B401FE56981
:10174F0070057F08027209E569B401057F0802720E
:0E175F001CE569B40207D22F7F06122C282247
:065433008F678D688B6994
:10543900E567703BE5687037E569700690000F0411
:105449008021E569B4010A90000F7402F0D22F801F
:1054590047E56964027041C21E7FFF1271C890005E
:105469000F7403F0C2307F02123160D22F8029E518
:105479006764017023E568701F7D077F0512519BE2
:105489005016E569700BC200C2307F03123160808B
:1054990007E569B40102D200302F0C90000FE0FD3E
:0754A9007F0F7E001266CAAE
:0154B00022D9
:105B63008F678D688B69E567700C125BA7749F2F35
:105B7300F58274008019E567B4010C125BA7749F6A
:105B83002FF58274008016E567B40209125BAF3EFD
:105B9300F583E4F022E567B40309125BAF3EF583B6
:105BA3007401F022AD69AF681271AC22AD69AF68C0
:0B5BB3001271AC746F2FF58274002299
:026C01008F679B
:106C0300AF057804EF08800123D8FD4BF568E567ED
:106C1300B40908E568B49903025223AD68AF67125B
:026C23006864A3
:016C2500224C
:0D71AC00EF75F00AA47C002DFFEC35F0FE1D
:0171B90022B3
:046A2B008F688D697A
:106A2F00C3E569648094E4501BE4F56AC3E56964C7
:106A3F0080F8E56A648098500BC22FAF68122C283B
:046A4F00056A80E86C
:016A53002220
:0D71BA00C296007F05126B6B126548D296DD
:0171C70022A5
:107051001271BAEF20E0F9C296007F06126B6BC283
:06706100B60000D29622E9
:107067001271BAEF20E0F9C296007F04126B6BC26F
:06707700B60000D29622D3
:046332008E608F6189
:10633600AE04AF058E638F64C296007F03126B6B4B
:10634600E560FF126B6BAF61126B6BE4F562126571
:1063560048E5642562F582E43563F583EFF005626E
:09636600E562C3942040E7D296E1
:01636F00220B
:085EE5008E658F668C678D68E5
:105EED001271BAEF20E0F985656A85666BC296007E
:105EFD007F02126B6BE567FF126B6BAF68126B6BFA
:105F0D00E4F569E56B2569F582E4356AF583E0FF13
:105F1D00126B6B0569E569C3942040E7C2B60000BA
:025F2D00D2960A
:015F2F00224F
:0A58C3008E5A8F5B8C5C8D5D8B5E4E
:1058CD00C2AF1270511271BAEF20E0F9855C60859C
:1058DD005D61C296007F02126B6BE55AFF126B6B16
:1058ED00AF5B126B6BE4F55FAF5EEF3395E0FEC31C
:1058FD00E55F9FEE6480F87480985014E561255F34
:10590D00F582E43560F583E0FF126B6B055F80D89F
:0B591D00C2B60000D296127067D2AF35
:01592800225C
:1066CA008E6B8F6C8D6DC2AF1270511271BAEF2042
:1066DA00E0F9C296007F02126B6BE56BFF126B6BDF
:1066EA00AF6C126B6BAF6D126B6BC2B60000D296B9
:0666FA00127067D2AF220E
:1063AD00C2AFE4F55BF55CF55DF55EF55FF55AAEF4
:1063BD005EAF5FAC5BAD5C1263327420255CF55C47
:1063CD00E4355BF55B7420255FF55FE4355EF55EC6
:0B63DD00055AE55AC3948940D6D2AFA0
:0163E8002292
:1060E500C2AF756200756300756400E4F560F56123
:1060F500F55F127051AE63AF64AC60AD61125EE5E1
:1061050074202561F561E43560F56074202564F53A
:1061150064E43563F563055FE55FC3948940D31295
:046125007067D2AF1E
:016129002253
:1059ED000500050105030507050F051F051E051C0F
:1059FD00051805100201040E040A03060101040B2B
:105A0D000304040F020304010302040D0200020249
:105A1D00030004090404030503070100030304073D
:105A2D00030104060402040C0516051500000615F5
:0E5A3D00062A060C06380633061E0612061749
:104FF4002430F58274003EF583EDFF3395E0FEE541
:10500400822FF582E5833EF583E0FFEDFB3395E0E7
:10501400FA22AF41126B6BC293127213D293D2AFC6
:10502400223EF583E0FC74B82FF582741D3EF583AF
:10503400ECF00D221528E528D394002225E024ED78
:10504400F582E43459F583E49322E4F57BD20EC26D
:1050540027C21DC21A227FA01271C8E4F542C21EE3
:1050640022127213D2B67801EF0822122EDAD2CAB3
:0F507400D20ED22722ECFF3395E0FEEF78032215
:1043EF00200E2F900540E004F576D3648094815021
:1043FF00030244AFD3E5766480948F400375760F44
:10440F00900029E0FF122EDA90002AE0F575125085
:10441F004E22301A5830271212503840030244AF40
:10442F00C2CAC227D21D85752822301D0A125038E4
:10443F00506EC227C21D22AF791579EF700BC21AC9
:10444F00E57525E0F528D21D22E57A30E005857562
:10445F00288008E57575F003A4F528AF7A7801EF89
:10446F0008800103D8FDF57AD227D2CA22D5760863
:10447F00C20EE4F542C21E22057B7440257BF582F5
:10448F00E43405F583E0125040540FF5797401932D
:10449F00F57A700AD21DE57525E025E0F528D21AC8
:0144AF0022EA
:1054B100200E12900029E0FF122EDA90002AE0F56A
:1054C1007712504E22301A5130270F125038505D4A
:1054D100C2CAC227D21D85772822301D0A12503830
:1054E100504BC227C21D22AF791579EF7007C21A3E
:1054F100C20EF54222E57A30E0058577288008E57D
:105501007775F003A4F528AF7A7801EF08800103DD
:10551100D8FDF57AD227D2CA22E543125040FA7457
:0D5521000193FBEA540FF579EBF57AD21AED
:01552E00225A
:10654800E4F56FD297F56E127213C2B6127213AFDA
:106558006F7801EF08800123D8FDF56F309703436A
:106568006F01127213D2B6127213056EC3E56E6410
:0765780080948840D2AF6F50
:01657F0022F9
:0972130000000000000000002250
:10698000C2B7E4FEC2B6127213EF30E704D2B5808C
:1069900002C2B5125065800123D8FDFF1272130E9A
:0B69A000BE08E1C2B6D2B7D2B6D2B535
:0169AB0022C9
:0D001600C2AFEF4227AF27126980D2AF22A0
:0E71C800C2AFEFF45227AF27126980D2AF2278
:106B6B00E4FEC2B6127213EF30E704D2B58002C254
:106B7B00B5125065800123D8FDFF1272130EBE08AB
:056B8B00E1D2B6D2B515
:016B900022E2
:09721C00C2AFEF424112501622EC
:0A720900C2AFEFF4524112501622FA
:102EDA00EF12126B2F42012F49022F50032F570472
:102EEA002F5E052F65062F6C072F73082F7A092F7F
:102EFA00810A2F880B2F8F0C2F960D2F9D0E2FA432
:102F0A000F2FAB102FB2112FB9122FC0132FC714C6
:102F1A002FCE152FD5162FDC172FE3182FEA192FCE
:102F2A00F11A2FF81B2FFF1C30011D30081E300F1D
:102F3A001F30162000002FFF75CB8E75CAC622756A
:102F4A00CB9575CA772275CB9B75CA692275CBA0BA
:102F5A0075CABA2275CBA675CA332275CBAB75CAA8
:102F6A00632275CBB075CA022275CBB475CAA32287
:102F7A0075CBB875CAFA2275CBBC75CAD82275CB7F
:102F8A00C075CAA82275CBC475CA362275CBC77557
:102F9A00CA862275CBCA75CABC2275CBCD75CAB48E
:102FAA002275CBD075CA762275CBD375CA302275F5
:102FBA00CBD575CAB22275CBD875CA132275CBDAAE
:102FCA0075CA522275CBDC75CA7D2275CBDD75CAEE
:102FDA006E2275CBE075CA542275CBE275CA1B22E4
:102FEA0075CBE375CAC32275CBE575CA5E2275CB6C
:102FFA00E675CADA22801C75CBE875CA902275CBB1
:10300A00EA75CAD92275CBEC75CA092275CBED755A
:0A301A00CA292275CBE875CA4122CD
:10002600C3EF648094A15008EF25E025E0F528226F
:04003600E4F52822A3
:023A49008F5A92
:103A4B00900118E0FFE55A7006E545D39F5012E54B
:103A5B005A64016003023B3FE546D39F5003023B90
:103A6B003FE55A7018C3E5459FF55D74602FF582ED
:103A7B00E4341EAD82F55E8D5F7F40801BE55AB44A
:103A8B000119C3E5469FF55D74B02FF582E4341E32
:103A9B00AF82F55E8F5F7F101200167FF47E0112EE
:103AAB006F6D7D207F051269D77D1A7F081269D74C
:103ABB007FC87E00126F6DE4F55BE55BC3955D50CF
:103ACB0061055FE55FAE5E7002055E14F5828E8365
:103ADB00E0F55C12126B3B1C003AFA0A3AFE0B3B08
:103AEB00040C3B0A0D3B100E3B160F00003B22E46F
:103AFB00FD80277D5F7F0780227D5E7F06801C7D9A
:103B0B000A7F0280167D327F0280107D467F028005
:103B1B000A7D0A7F038004AD5CE4FF1269D7055B65
:103B2B008098E55A70047F408007E55AB401057F01
:043B3B00101271C82B
:013B3F002263
:10533000200E10754406901DB8E06003D20E22E4E2
:10534000F54222E528D394004003152822C2CA154D
:1053500044E54414603D14603214601D146015145B
:105360007049901DB8E0FF7003F54222122EDA90CA
:105370001DB9802F901DBA8015901DBBE0FF7003F2
:10538000F54222122EDA901DBC8018901DBDE0FF60
:10539000020026901DBEE0FF7003F54222122EDAB5
:1053A000901DBFE0FF120026D2CA22E4F542C2CA15
:0353B000C20E2208
:10695200900028E0FF6026200E0712506F75281461
:1069620022E528D394004003152822202708D2CA02
:0E697200752814D22722C2CA75287DC227229A
:1068F400200E0C7F1C12506F75286475783C22E5BD
:1069040028D394004003152822AF781578D3EF6478
:0E691400809480400475286422C20EE4F5428F
:016922002252
:10662700E54214601C14601C14601F14602214607F
:106637002224057021C2CAC20EC227C21DE4F54436
:1066470022025330126952D21E221243EFD21E2267
:076657000268F41254B122A5
:10676A00BF010790002A7418F022BF020790002A7E
:10677A007412F022BF030590002A8014BF04079008
:10678A00002A740BF02290002ABF05047409F02233
:04679A00740CF02269
:0252AA00AC074F
:1052AC00C3EC64809480404AEC6480948850432022
:1052BC002B21E4FD125079C333CE33CED8F9124FE3
:1052CC00F474102BF58274003AF583EFF00DBD08E1
:1052DC00E3801FE4FD125079C333CE33CED8F912DC
:1052EC004FF474182BF58274003AF583EFF00DBD72
:1052FC0008E3202B16E4FDEDFF3395E0FE74102F30
:10530C00F5827400125025BD08ED22302B15E4FDFA
:10531C00EDFF3395E0FE74182FF5827400125025C2
:03532C00BD08EDCC
:01532F00225B
:105223007D3F7F091269D77D507F081269D790723D
:10523300451252A17D5B7F061269D79072461252C6
:10524300A1907247E493FDE4FF1269D7907248E49A
:105253009312126B527341527742527B43528144F1
:10526300528745528D46529347529948000052A0A7
:105273007D0A80067D3280027D467F02801C7D0A86
:105283007F0380167D287F0380107D467F03800A7D
:105293007D0A7F0480047D287F041269D722E4936A
:0752A300FDE4FF1269D722B0
:106274008F5BE55B7005D22DFF8009E55BB40107F8
:10628400D22D7F01125CC77D4B7F021269D77D023C
:10629400E4FF1269D77D32E4FF1269D7125223E575
:1062A4005B70028005E55BB401057F401271C82272
:103FBF00A209300501B350307D017F0412519B508F
:103FCF002320050E30090B9000A4E0FF7C0B7D60D1
:103FDF00800F30050F20090C9000A5E0FF7C0B7DB2
:103FEF0080125E9AA2099205A20A300601B35030E0
:103FFF007D027F0412519B502320060E300A0B9036
:10400F0000A6E0FF7C0B7DA0800F30060F200A0C6E
:10401F009000A7E0FF7C0B7DC0125E9AA20A920669
:10402F00A20B300701B350307D037F0412519B5018
:10403F002320070E300B0B9000A8E0FF7C0B7DE0D8
:10404F00800F30070F200B0C9000A9E0FF7C0C7D38
:10405F0000125E9AA20B9207A20D300801B35030E6
:10406F007D047F0412519B502320080E300D0B90BE
:10407F0000AAE0FF7C0C7D20800F30080F200D0C74
:10408F009000ABE0FF7C0C7D40125E9AA20D92086F
:01409F0022FE
:10683400534103900024E0FE543FFF780408800194
:1068440023D8FD54F0FFEE30E40343070490002402
:0F685400E030E503430708EF4241C2AF12501690
:016863002212
:022C28008F6BB0
:102C2A00302F05756CF48003756C64E56B64017074
:102C3A0029AF417803EF08800123D8FD3392307F12
:102C4A001020300B122D447F10127209022D3C12F3
:102C5A002D4F7F1012721C022D3CE56B6402702806
:102C6A00AF417802EF08800123D8FD3392307F20EC
:102C7A0020300A122D447F201272098008122D4F2B
:102C8A007F2012721C022D3CE56B64037028AF4151
:102C9A007801EF08800123D8FD3392307F4020303D
:102CAA000A122D5A7F401272098008122D657F4040
:102CBA0012721C022D3CE56B6404701EE5413392CE
:102CCA00307F8020300A122D5A7F801272098008C4
:102CDA00122D657F8012721C8058E56B640570277F
:102CEA00AF417805EF08800123D8FD3392307F0485
:102CFA0020300A122D707F041272098008122D7B6F
:102D0A007F0412721C802BE56B6406702CAF41782D
:102D1A0004EF08800123D8FD3392307F0820300A5F
:102D2A00122D707F081272098008122D7B7F0812FB
:092D3A00721CAF6C7E00126F6D7B
:102D43002212721CAF6C7E00126F6D22127209AFD9
:102D53006C7E00126F6D2212721CAF6C7E00126FBC
:102D63006D22127209AF6C7E00126F6D2212721CFB
:102D7300AF6C7E00126F6D22127209AF6C7E00126F
:032D83006F6D224F
:10600D00900024E030E0057F1012721C900024E017
:10601D0030E1057F2012721C900024E030E2057FF4
:10602D004012721C900024E030E3057F8012721C38
:10603D00900024E030E4057F0412721C900024E0EF
:09604D0030E5057F0812721C22E7
:106FBE0030030A12505AC203C211C21E22300409F3
:0A6FCE0012505AC204C213C21E2260
:106864008F708D71E570B4011FE5717003125F3094
:10687400E571B40107787FE6FF125D6AE571B43211
:106884000E7FF47E01026F6DAD71AF701269D72275
:1069D700EFFEEDFF1280008E2D8F2E1256977574E5
:1069E70032AF741574EFD39400400EE4F573E5737A
:0969F700C3943A50EC057380F5DD
:016A00002273
:10569700D2A8AFA875A881C214852E82852D83E470
:1056A70093C4540FFE4306F08E80C284D28500C295
:1056B700870000D287007580FF7580FEC284C2858F
:1056C70000C2870000D287007580FFD2147D407C1E
:1056D7001FE4FE30B40D0EBE32F9ED1D70011CED56
:1056E7004C70EE7C1F7D40E4FE20B40D0EBE32F9F7
:1056F700ED1D70011CED4C70EE8FA8C2A87F0A7ECD
:0457070000126F6DB0
:01570B00227B
:106A01007580FDC284C28500C28700000000D28764
:106A1100007580FF7F0A7E00126F6D7F997E0912DB
:0A6A210080008E2D8F2E1256972252
:1044B000D284D285C286A2809217A2819220A28243
:1044C0009218A2839221D2862001537D027F01128D
:1044D000519B40137D037F0112519B400A30170707
:1044E000301932D22480377D027F0112519B500F48
:1044F00030170C302009301904D224802180167D19
:10450000037F0112519B501220170330200C3019E9
:1045100004D2248009126AA58004C219C224200290
:104520004E7D027F0212519B40127D037F02125189
:104530009B4009301806301B2FD225227D027F02B6
:1045400012519B500E30180B302108301B03D2251E
:104550002280157D037F0212519B500F20180330DB
:104560002109301B03D22522026ACDC21BC225229B
:106AA500753D1E753E60E4FFE53E2FF582E4353DFC
:106AB500F583E4F00FBF50F0753D1E753E60E4F5BB
:076AC50045C226C211D219DF
:016ACC0022A7
:106ACD00753F1E7540B0E4FFE5402FF582E4353F7C
:106ADD00F583E4F00FBF10F0753F1E7540B0E4F57F
:076AED0046C228C213D21BB0
:016AF400227F
:106EFB00C284D285C286A2809209A281920AA28202
:0D6F0B00920BA283920DD286D284D28522F1
:10642500E57D2560F582E4357CF5832274FF121243
:1064350041E4FBFAF9F8C302122E057E7480257D2E
:10644500F57DE4357CF57C22F582E4341DF5832267
:0B645500757E01757C00757D20E4223F
:104570007D027F0712519B50057F04127209C229E8
:10458000D223E4F5427FE87E03126F6DC298C2AF7A
:10459000C2307F03123160755E7F755D96755C98E1
:1045A000755B00785B126431504430983E1200060F
:1045B00012711FEF14601824F0602624C1600B24D0
:1045C000F670287F0612722E802112650F801C7FE4
:1045D0000612722E126CD91268341260E5D229804C
:1045E0000A7F0612722E125D1AD2293029B5E4789C
:1045F00084F6D2307F011231607F40120016C22F44
:10460000126C937D467F021269D77D1E7F07126967
:10461000D77D147F081269D77D327F031269D7C214
:0D462000307F031231607FFF1271C8C2238A
:01462D00226A
:105D1A00126455F55F7F0212722EE57E2402F56148
:105D2A00AF7E12722EE4F560126425E0FF12722E25
:105D3A00126425E02561F5610560E560C394804041
:105D4A00E7AF6112722E7F0312722E12609EEF6409
:0F5D5A0015600C12643F055FE55FC3942240B6ED
:015D69002217
:106CD900126455F55F12679E50077F0612722E8067
:106CE900057F1502722E12643F055FE55FC394228A
:026CF90040E376
:016CFB002276
:10679E00E4F56012723674D0256012644DEFF00588
:1067AE0060E560C3948440EB1270FD901E52E0B51C
:1067BE000710AE7CAF7DBE0504BF200100126F51E5
:0367CE00D322C310
:0167D10022A5
:106F5100E4FF74D22FF582E4341DF583E0FEE57D74
:0B6F61002F126429EEF0000FBF80E744
:016F6C002202
:1070FD00E4FFFE74D02E12644DE02FFF0EBE82F31E
:01710D00225F
:10650F00E4F55FF5657564E0756393756204F56195
:10651F00786112643150213098F61200068F60E5D1
:10652F006064046013AF65056574D02F12644DE588
:08653F0060F0255FF55F80D8D4
:016547002231
:04000600AF99C29854
:01000A0022D3
:08722E003099FDC2998F9922ED
:077236003098FDAF99C298EA
:01723D00222E
:10609E00E4F565F564F563F5627F007EE87D7D7C51
:1060AE0047AB65AA64A963A8621210EE502430981B
:1060BE0005C298AF9922AF65AE64AD63AC62E4FBE6
:1060CE00FA7980783F120FFD8F658E648D638C6236
:0660DE0080C7C2987F009C
:0160E4002299
:10700B000C0102030405060708090A0B0C01020315
:08701B000405060708090A0B31
:106A5400AF5FEF3395E0FE75F007EF12125FEE754E
:106A6400F007A42583F583E0227882E6FF126FF213
:096A7400EF22C295D297D2AF22A5
:106B9100C22CC2AF12723E7F83127023126E0A1290
:106BA1006A767883E66F600B1261B0302B05126252
:056BB100B4922CA22C9F
:016BB60022BC
:1062B4007983E778866660367883E6FF7886F6EF3A
:1062C4007013E552C3940A500C7D077F0412519B4E
:1062D400500312612A7D057F0412519B5010E54141
:1062E40054036005124180D322124180C322C32289
:10418000E4F55F900A50126A547003024244900AA8
:1041900051126A5B60167880666003024244900A9E
:1041A00052126A547887666003024244AF5FEF336D
:1041B00095E0FE900A53126A5BFF787FE6FEEF6E91
:1041C0006020EF601DB4080BEED394014005EE941F
:1041D00007400FEF6409706CEE64016005EE640740
:1041E0007062AF5FEF3395E0FE900A54126A5BFF96
:1041F000F46006EF788266704BE55FFD3395E0FC76
:10420000900A5575F007ED12125FEC126A6378831D
:10421000667031D201D20274BD2DF58274003CF576
:1042200083E0FFC007EDAE047805C333CE33CED8AC
:10423000F92480F582740E3EAD82FCD007125E9A9E
:10424000C201C202055FC3E55F648094935003021C
:024250004183A8
:014252002249
:10612A007D087F0412519B500D7882E6FF126FF2B0
:10613A00EFC39407402CD2307F011231607F4012A6
:10614A000016C22F126C93D201D202E4FD7F0A120A
:10615A004BC9C201C2027F501271C8C2307F0112FC
:03616A003160227F
:1061B000C2AF12723E7FBF127023126E0A7883A69E
:1061C00007126E0A7883A607126E0A7882A6071253
:1061D0006E0A7887A607126E0A7880A607126E0AE2
:1061E000787FA607126E0A7881A60712723E126A9D
:0261F000762215
:105BBE00C2AF12723E7F8E125C0D7F901270237FE9
:105BCE00A712702312723E7FBE127023E4FF127072
:105BDE00237883E6FF1270237882E6FF1270237813
:105BEE0087E6FF1270237880E6FF127023787FE637
:105BFE00FF1270237881E6FF125C0D126A76221274
:0B5C0E007023E4FF12702312723E228C
:105D6A008F72E572B401047D63803EE572B4020667
:105D7A007D087F068035E572B403067D317F088091
:105D8A002AE572B404067D617F08801FE572B405B6
:105D9A00067D257F088014E572B406067D597F03C7
:0F5DAA008009E572B407077D487F071269D72289
:026FF200AE07E8
:106FF400EE54F0FF780408800103D8FD75F00AA46C
:06700400FFEE540F2FFF08
:01700A002263
:105F3000126A6D90700B93FF12384E7883126A6F5D
:105F4000601B7883126A6FC3940A50077D327F0604
:105F50001269D77883E6FF126FF212384E126A6D1B
:105F6000C3940C50067D0A7F0280047D507F061288
:0A5F700069D77D507F051269D72222
:105C71007FF47E01126F6D7D097F061269D77880EE
:105C8100125CB77D0E7F031269D77D357F061269DD
:105C9100D77D097F061269D77887125CB77D1E7F91
:105CA100091269D77D1E7F071269D77881E6FF1235
:105CB1006FF212384E22E6FF126FF212384E7FF465
:065CC1007E01126F6D224E
:07723E00C2B6C295D29522F1
:10702300E4FEC297EF30E002D297C2B6D2B6EFC306
:0670330013FF0EBE08EC85
:017039002234
:106E0A00E4FFD297FED2B6C2B6A297E433C43333B4
:0F6E1A00335480FDEFC313FFED42070EBE08E6B1
:016E29002246
:105B0600EF3395E0FE74702FF58274003EF583E066
:105B1600FF22AF5AEF3395E0FEEF222460F5827440
:105B2600013EAD82FCD22922900520E0F547A3E094
:105B3600F548222450F58274053EAD82FC22900081
:105B4600BAE0FF7C0E7D2022D222D201E4FF22C2DF
:0D5B560001C2227F1922D222D2307F02220A
:102AC700E55270081271F28F52022BC2E552B4051B
:102AD700081247A08F52022BC2E552B40B08126F9F
:102AE700888F52022BC2E552B40A08125F7A8F52BE
:102AF700022BC2E552B40F0812616D8F52022BC22E
:102B0700E552B414081225D68F52022BC2E552B4EF
:102B17001908126E678F52022BC2E552B41E0812B3
:102B27006D428F52022BC2E552B42308126DA88F53
:102B370052022BC2E552B428071271D68F52807BFE
:102B4700E552B42D07126B1D8F52806FE552B432D8
:102B5700071265808F528063E552B43E07126E8577
:102B67008F528057E552B43C071270C78F52804B83
:102B7700E552B43307126D868F52803FE552B44158
:102B8700071271508F528033E552B44C07127160AF
:102B97008F528027E552B444071271708F52801B01
:102BA700E552B4370712598E8F52800FE552B43968
:102BB7000712570C8F528003E4F552E55370061243
:102BC700000E8F5322E553B405061272258F532248
:102BD700E553B40A061271808F5322E553B40F06EA
:102BE70012718F8F5322E553B41406123DFB8F5396
:102BF70022E553B43D06126EA38F5322E553B43F2B
:102C0700061268948F5322E553B44306126AF58F70
:102C17005322E553B44D06126DC98F5322E4F55381
:012C2700228A
:0D71F20090052AE0F52BA3E0F52C7F052287
:1047A000302414201011C21C7D047F0112519B5033
:1047B000037F0B227F0A227F0812665E5006124991
:1047C0000B7F0022202408301005C2107F05227DB7
:1047D000057F0612519B501EE53945387018900030
:1047E000B5E0FF7C0D7D80125E9A90052EE0F538D5
:1047F000A3E0F53980517D067F0612519B501EE5DE
:104800003C453B70189000B6E0FF7C0D7DA0125E29
:104810009A900530E0F53BA3E0F53C802A7D077FC8
:104820000512519B500B300008E52C452B7002C23D
:1048300000300F08E52C452B7002C20F7884E6B4D7
:1048400005057F0412552FE551700875510AD22BCA
:06485000126B917F0522AE
:106F8800200F1590053BE0F54E2024037F0522E5F0
:0B6F98004ED3940050F3D20F7F0A226A
:105F7A007D077F0512519B500C7D077F0512519BAF
:105F8A00503230002F7D017F0112519B5026D230B2
:105F9A007F011231607F011200167D027F071251C4
:105FAA009B50057F0412721C9000A0E0FF7C0A7DC2
:0A5FBA00E0125E9A125B2E7F0F22A8
:10616D0030243DE5484547700C7D087F0112519B59
:10617D0050037F372230030EE53A700A126FBE7F4F
:10618D000112001680173026037F14227884E6B49E
:10619D00050B7F0312552F2024037F14227F0F221E
:0361AD007F14223A
:1025D60090053DE0F54B7F011271C8126FBE7D027A
:1025E6007F0712519B5009E54B70057F0412720953
:1025F6009000A1E0FF7C0B7D00125E9AD22B126B3D
:1026060091E54570030227007C017D001227885062
:10261600037F3E227C017D5012276850037F3C22B7
:102626007C017D5812276850037F3C227C017D1077
:10263600122770500812277850037F33227C017DC1
:1026460020122770500B9000BBE0FF7C0E7D40806F
:10265600207C017D281227805005125B4480127C65
:10266600017D3012278050129000B9E0FF7C0E7D6C
:1026760000125E9A126AA57F00227C017D40D22953
:10268600E4FF124B20500C7D067F0412519B500331
:102696007F4C227C017D3812278850037F44227CA0
:1026A600017D18C229E4FF124B20500C7D057F01E5
:1026B60012519B50037F4122E4F55A125B187803AE
:1026C600C333CE33CED8F9125B21E4FF124B205030
:1026D6001BAF5A125B06C007125B187805C333CED0
:1026E60033CED8F9125B39D007125E4F055AC3E5CF
:1026F6005A648094A840C47F1922122778500C7D12
:10270600077F0512519B504B3000487884E67004D1
:102716007F0180087884E6B404077F0212552F8073
:102726002F7884E6B40704760180257D037F0612A0
:10273600519B501CE557455670169000AFE0FF7C44
:102746000C7DC0125E9A900532E0F556A3E0F5576F
:102756007F19227D077F0512519B50052000027FBD
:01276600056D
:1027670022D229E4FF124B2022D229E4FF124B2068
:10277700227D077F0512519B22D229E4FF124B20AD
:0927870022C229E4FF124B2022BA
:106E6700302603126AA57D077F0512519B50062025
:0E6E770000037F0522900538E0F54E7F1E22B5
:106D4200E54E70037F23227D027F0712519B50097B
:106D5200E54B70057F041272093024037F0A227FFB
:026D62001E22EF
:106DA800125B2E7D067F0112519B500C9000ACE0C7
:106DB800FF7C0C7D60125E9A900539E0F54E7F2DC0
:016DC80022A8
:0E71D6007FA01271C8900539E0F54E7F2D2282
:106B1D00D22B126B917D027F0712519B5009E54BD1
:106B2D0070057F04127209E54E70037F3222302406
:076B3D00037F0A227F2D22D5
:10658000301E037F32227D047F0612519B501FE58F
:1065900055455470199000B0E0FF7C0C7DE0125E10
:1065A0009A900534E0F554A3E0F5557F3222C230CD
:0865B0007F011231607F00221F
:1070C70020220CD222E4FF120556C2227F00227F23
:0270D7003C2259
:106E8500202218D2227F40120016D20112201DC2E4
:0E6E9500017F401271C8C2227F19227F3E2267
:1071500020220A125B4E123A49125B55227F4122CD
:1071600020220A125B4E1263E9125B55227F4422F1
:1071700020220A125B4E12577C125B55227F44225A
:05000E0000007F052247
:097225003025037F0A227F0522B7
:0F7180009000A2E0FF7C0B7D20125E9A7F0F2211
:0F718F003025093028037F14227F0F227F14221E
:103DFB009000A3E0FF7C0B7D40125E9AE5467003BA
:103E0B00023ED37D017F0312519B50707C017D08D4
:103E1B00C2297F01124B2050037F3F227C017D5032
:103E2B00123ED650037F3D227C017D58123ED65068
:103E3B00037F3D227C017D40D2297F01124B205014
:103E4B000C7D067F0412519B50037F4D227C017D1C
:103E5B0028D2297F01124B205009125B44125E9A23
:103E6B007F00227C017D18C2297F01124B20500C50
:103E7B007D057F0212519B50037F43227D027F03FE
:103E8B0012519B5043E4F55AAF5A125B1A7803C395
:103E9B0033CE33CED8F9125B217F01124B20501D4C
:103EAB00AF5A125B06C007AF5A125B1A7805C333C1
:103EBB00CE33CED8F9125B39D007125E4F055AC3F9
:0A3ECB00E55A648094A840C07F000F
:093ED50022D2297F01124B2022A8
:106EA300202218D222C2307F011231607F01127179
:0E6EB300C87F01120556C2227F00227F3D22B9
:1068940020222A125B5C1231607FF47E01126F6D3C
:1068A4007F10120016D202121E1CC2027F10127137
:1068B400C8C2307F02123160C2227F00227F3F2291
:106AF500202222125B5C1231607FF47E01126F6DE1
:106B0500D2027F01123A49C202C2307F02123160BD
:086B1500C2227F00227F43220F
:106DC90020221B125B5C123160D2027F011263E93F
:106DD900C202C2307F02123160C2227F00227F4D7F
:016DE9002287
:1057EA00AF5AEF3395E0FE22900520E0F547A3E09B
:1057FA00F54822900522E0F549A3E0F54A22246003
:10580A00F58274013EAD82FCD2292274702FF58292
:10581A0074003EF583E0FF22C202C2227F192224CD
:10582A0050F58274053EAD82FC22900536E0F532D1
:10583A00A3E0F53322055AC3E55A648094A822D21C
:0D584A0022C2307F0122D222C2307F022212
:1034FB00E5527006126D648F5222E552B405061226
:10350B00394D8F5222E552B40B06126B448F522267
:10351B00E552B40A0612462E8F5222E552B40F061C
:10352B001270D98F5222E552B41106125A4B8F5298
:10353B0022E552B412061253B38F5222E552B41441
:10354B0006120A4F8F5222E552B419061269238FC5
:10355B005222E552B41E061268C48F5222E552B4B1
:10356B0023061262338F5222E552B428061271E4FD
:10357B008F5222E552B42D061264608F5222E5520F
:10358B00B432061265B88F5222E552B43C06127063
:10359B00EB8F5222E552B43D06126FA38F5222E5F8
:1035AB0052B43E06126C268F5222E552B43F0612DD
:1035BB00710E8F5222E552B44106126E2A8F52229F
:1035CB00E552B44306126CFC8F5222E552B44C0602
:1035DB00126FD88F5222E552B44D06126D1F8F52C7
:1035EB0022E552B4370612598E8F5222E552B43966
:1035FB000612570C8F5222E552B438061269AC8F63
:10360B005222E552B43306126D868F5222E552B424
:0C361B00440612703A8F5222E4F552224D
:106D640090052AE0F52BA3E0F52C7D067F02125155
:106D74009B500C90052CE0F529A3E0F52AD21F7F47
:026D84000522E6
:10394D00302414201011C21C7D047F0112519B5094
:10395D00037F0B227F0A22302514201211D21C7DE9
:10396D00047F0212519B50037F0B227F0A227F0896
:10397D0012665E500612490B7F002220240830107B
:10398D0005C2107F0522202508301205C2127F05C1
:10399D00227D057F0612519B501EE5394538701862
:1039AD009000B5E0FF7C0D7D80125E9A90052EE0B3
:1039BD00F538A3E0F53980757D067F0612519B50D1
:1039CD001EE53C453B70189000B6E0FF7C0D7DA0D8
:1039DD00125E9A900530E0F53BA3E0F53C804E7DFC
:1039ED00077F0512519B500D30000AE52C452B70B9
:1039FD0004C200800B300F08E52C452B7002C20F5E
:103A0D007D067F0212519B5019301F16E52A45295C
:103A1D007010C21F9000BCE0FF7C0E7D60125E9A9C
:103A2D00800B7884E6B405057F0412552FE551709F
:0C3A3D000875510AD22B126B917F0522F4
:106B4400200F2190053BE0F54E202406201C037FF6
:106B54000522202506301C037F0522E54ED3940030
:076B640050E7D20F7F0A2267
:10462E007D077F0512519B50127D077F0512519B0E
:10463E0040030246DF2000030246DF201C3FD2303B
:10464E007F031231607F0F1271C890000FE0B40229
:10465E00047F05800990000FE0B403057F0112006E
:10466E00161257F27D027F0712519B50057F0412DE
:10467E00721C9000A0E0FF7C0A7DE0804E301C5141
:10468E0090000FE0FF64026005EF640370437F0F3C
:10469E001271C87F0512665E400BD2307F01123157
:1046AE00607F028009D2307F031231607F0A1200D0
:1046BE00167D027F0712519B50057F0412721C1249
:1046CE0057FD9000A2E0FF7C0B7D20125E9A7F0FBB
:0A46DE00221257F21257FD7F0F223F
:1070D900201C063024037F1122301C053025027F35
:0270E900122271
:105A4B00302458E5484547700C7D087F0112519B67
:105A5B0050037F3722300329E53A70257FA012715E
:105A6B00C890000FE0B401047F01800990000FE0A3
:105A7B00B402057F05120016E4F542C21EC2038074
:105A8B00173026037F14227884E6B4050B7F0312AC
:0E5A9B00552F2024037F14227F11227F142216
:1053B300301C1030240D20100A7F0A1271C8C21C41
:1053C3007F0A22301C5230254F20124C3003031227
:1053D3006FBEE54A4549700C7D087F0212519B5010
:1053E300037F3822300417E53A70137FA01271C887
:1053F3007F02120016E4F542C21EC2048017302851
:10540300037F14227884E6B4050B7F0312552F2003
:1054130025037F14227F1222201C1230250F201215
:105423000CD21CC2307F021231607F0A227F142209
:100A4F0090053DE0F54B7F0F1271C8201C0C9000F4
:100A5F00A1E0FF7C0B7D00125E9A301C0C9000A36E
:100A6F00E0FF7C0B7D40125E9AE542B403037F14D6
:100A7F0022126FBEE4F5427D027F0712519B50098F
:100A8F00E54B70057F04127209D22B126B91301C4B
:100A9F0003020B92E5457003020B927C017D00125D
:100AAF000D1950037F3E227C017D50120CE950033B
:100ABF007F3C227C017D58120CE950037F3C227C45
:100ACF00017D10120CF15008120D0150037F3322DB
:100ADF007C017D20120CF15003020BF97C017D2863
:100AEF00120D09500C9000BAE0FF7C0E7D20020C15
:100AFF00027C017D30120D09500C9000B9E0FF7C93
:100B0F000E7D00020C027C017D40D229E4FF124BC6
:100B1F0020500C7D067F0412519B50037F4C227C8A
:100B2F00017D38120D1950037F44227C017D18C2BC
:100B3F0029E4FF124B20500C7D057F0112519B5071
:100B4F00037F4122E4F55A1257EAEF7803C333CEFD
:100B5F0033CED8F9125808E4FF124B20501D12570C
:100B6F00EA125815C0071257EAEF7805C333CE3390
:100B7F00CED8F9125829D007125E4F12583F40C7EE
:100B8F007F1922201C03020C85E5467003020C8599
:100B9F007D017F0312519B4003020C3D7C017D08B8
:100BAF00C2297F01124B20500F7F50120016D230F6
:100BBF007F021231607F3F227C017D50120CF95071
:100BCF00037F3D227C017D58120CF950037F3D229B
:100BDF007C017D10120D115008120D0150037F334F
:100BEF00227C017D20120D1150129000BBE0FF7C82
:100BFF000E7D40125E9A126AA57F00227C017D4015
:100C0F00D2297F01124B20500C7D067F0412519B7D
:100C1F0050037F4D227C017D18C2297F01124B208A
:100C2F00500C7D057F0212519B50037F43227D02A2
:100C3F007F0312519B503CE4F55A1257EAEF7803A9
:100C4F00C333CE33CED8F91258087F01124B205040
:100C5F001D1257EA125815C0071257EAEF7805C34D
:100C6F0033CE33CED8F9125829D007125E4F12580F
:100C7F003F40C77F1922120D215008120D21504BF2
:100C8F003000487884E670047F0180087884E6B4E9
:100C9F0004077F0212552F802F7884E6B40704765D
:100CAF000180257D037F0612519B501CE557455649
:100CBF0070169000AFE0FF7C0C7DC0125E9A90051D
:100CCF0032E0F556A3E0F5577F19227D077F051215
:090CDF00519B50052000027F0525
:100CE80022D229E4FF124B2022D229E4FF124B2002
:100CF80022D2297F01124B20227D077F0512519BAA
:100D080022D229E4FF124B2022D2297F01124B2044
:100D180022C229E4FF124B20227D077F0512519B36
:010D280022A8
:10692300C219C2307F02123160302605126AA58077
:1069330006302803126ACD7D077F0512519B50064E
:0F6943002000037F0522900538E0F54E7F1E22CD
:1068C400E54E70037F23227D027F0712519B5009FE
:1068D400E54B70057F041272093024062010037FF3
:1068E4000A22302508201205D21C7F0A227F1E228C
:10623300201C051257F280031257FD7D067F0112C1
:10624300519B5024E5427020201C0B9000ACE0FFD2
:106253007C0C7D60800C301C0C9000ADE0FF7C0C4E
:106263007D80125E9A7F2822900539E0F54E7F2DBE
:016273002208
:0E71E4007FA01271C8900539E0F54E7F2D2274
:10646000D22B126B917D027F0712519B5009E54B95
:1064700070057F04127209E54E601D30240620105D
:10648000037F0A2290000FE0640160093025062096
:0B64900012037F05227F2D227F3222A5
:1065B800301E037F32227D047F0612519B501FE557
:1065C80055455470199000B0E0FF7C0C7DE0125ED8
:1065D8009A900534E0F554A3E0F5557F3222C23095
:0865E8007F011231607F0022E7
:1070EB0020220CD222E4FF120556C2227F00227FFF
:0270FB003C2235
:106C260020221FC2307F02123160D2227F40120022
:106C360016D20112201DC2017F401271C8C2227FE6
:056C460019227F3E222F
:10710E0020220BD222D202121E1C125822227F3FA4
:01711E00224E
:106FA3002022151258491231607F401271C87F01A7
:0B6FB300120556C2227F00227F3D2203
:106E2A002022191258501231607F101271C8D201F3
:0F6E3A00E4FF123A49C201C2227F19227F41228E
:106CFC0020221D1258491231607F401271C8D230C7
:106D0C007F02123160D2027F01123A4912582222BC
:036D1C007F432290
:106FD800202214125850123160D201E4FF1263E9E2
:0A6FE800C201C2227F19227F41225C
:106D1F0020221D1258491231607F401271C8D230A3
:106D2F007F02123160D2027F011263E912582222D0
:036D3F007F43226D
:10703A00202211125850123160D202E4FF12577CFA
:07704A00125822227F4422AC
:10598E00D2107D027F0712519B50057F04127209BF
:10599E0090000FE0FF64016004EFB4030E7F01126C
:1059AE0071C87F401259DD7F01801390000FE0B463
:1059BE00020F7F051271C87F501259DD7F031272DC
:1059CE00097F501271C83015031258347F392212D4
:0F59DE000016C22F126C93E4FD7F07124BC922F3
:10570C0030241130150BE53345327005C231126C63
:10571C004B7F3922E47884F6C21090000FE0FF64CE
:10572C00016005EF64037010D2307F011231607F8D
:10573C004012576A7F01801B90000FE064027016C4
:10574C00D2307F031231607F051271C87F5012571F
:10575C006A7F031231607F501271C87F00221200E1
:10576C0016C22F126C93E4FD7F08124BC9C2302273
:1069AC00D2127F0A1271C87F40120016D22F126CBD
:1069BC0093E4FD7F07124BC97F031272097F5012BB
:0B69CC0071C83015031258347F002200
:106D860030000B9000B8E0FF7C0D7DE0800C200009
:106D96000E9000B7E0FF7C0D7DC0125E9AB2007FB8
:026DA6001922B0
:1063E9008F5AE55A24FF922F126C93E55A70127F47
:1063F90040120016D201E4FD7F09124BC9C2018087
:1064090015E55AB401107F10120016D202E4FD7F7F
:0C64190009124BC9C2027F501271C82248
:10425300900540E07003024316C201C202D20C7FF4
:10426300501271C87F8012001675420390000FE050
:10427300640170323024297F011200167D027F070A
:1042830012519B50057F0412721C302404E54270C6
:10429300F920240C7F0112431A50057F041272097E
:1042A300E54270D0806490000FE0FF64026005EF88
:1042B300640370563024357F021271C87F051200E3
:1042C300167F0212721C7D027F0712519B50057FDD
:1042D3000412721C302404E54270F92024287F055F
:1042E30012431A50217F04127209801A3025177F56
:1042F30002120016202407302504E54270F620251B
:10430300057F021271C8E54270AA7FA01271C8C26C
:104313000CC21EE4F542221271C87D027F071251BE
:024323009B22DB
:03000000026F1874
:106F1800758E0078FEE4F6D8FD9000007FFF7E1F96
:0D6F2800E4F0A3DFFCDEFA758187024F6400
:100FF600021190E86480F8E933E83360110460F088
:10100600ED33EC337009E8FCE9FDEAFEEBFF220460
:1010160060DED3EB9FEA9EE99DE8C2E78CF0C2F75B
:1010260095F0400CE8CCF8E9CDF9EACEFAEBCFFB27
:1010360012115B85D0F05804700320D5B3E8047014
:10104600075002B2D502119A92D5EC0460F7E4CCAF
:10105600C0E0C398F8603B94186008400DD0E0FBF0
:10106600021172E4FBFAC9FC8028E830E406E4C900
:10107600FBE4CAFCE830E305E4C9CACBFCE8540744
:101086006010F8C3E913F9EA13FAEB13FBEC13FC4F
:10109600D8F130F52FC3E49CFCEF9BFFEE9AFEEDF2
:1010A60099FDD0E0FBEF4E4D4C701222DB0302118E
:1010B60097EC2CFCEF33FFEE33FEED33FDED30E71E
:1010C600EB021172EF2BFFEE3AFEED39FDD0E0FB9D
:1010D60050130BBB000302119AED13FDEE13FEEF46
:0810E60013FFEC13FC02117270
:1010EE0074F8CC6480CCC86480C8F582046043C3B5
:1010FE00EB9FF5F0EA9E42F0E99D42F0E89C45F048
:10110E0060305018E5825FFFE582F42B5582FB506C
:10111E00210ABA001D09B90019088016E5825BFB89
:10112E00E582F42F5582FF50090EBE00050DBD005D
:10113E00010CC3EB9FF5F0EA9E42F0E99D42F0E808
:0D114E009C45F06007CC4820E701B3EC227F
:10115B00E9D2E7C933E833F892D5EDD2E7CD33ECDA
:07116B0033FC5002B2D52253
:10117200EC30E7100FBF000C0EBE00080DBD0004DE
:101182000BEB6014A2D5EB13FCED92E7FD2274FF8A
:10119200FCFDFEFF22E480F8A2D574FF13FC7D80E3
:0311A200E480EFF7
:1011A500C2D530F707B2D563F0FF05F030E70CB2D2
:1011B500D5F4048463F0FF05F080018430D502F492
:0211C500042202
:1011C700EF8DF0A4A8F0CF8CF0A428CE8DF0A42E3C
:0211D700FE22F6
:1011D900BC000BBE0029EF8DF084FFADF022E4CCFA
:1011E900F875F008EF2FFFEE33FEEC33FCEE9DECC3
:1011F900984005FCEE9DFE0FD5F0E9E4CEFD22ED09
:10120900F8F5F0EE8420D21CFEADF075F008EF2F52
:10121900FFED33FD4007985006D5F0F222C398FD43
:051229000FD5F0EA22E0
:10122E00EB9FF5F0EA9E42F0E99D42F0E89C45F016
:01123E00228D
:10123F007401FF3395E0FEFDFC080808E6CF2FF69A
:10124F0018E6CE3EF618E6CD3DF618E6CC3CF62273
:0C125F00A42582F582E5F03583F583229A
:10126B00D083D082F8E4937012740193700DA3A312
:10127B0093F8740193F5828883E473740293686026
:06128B00EFA3A3A380DF26
:10711F00EFC39461400AEF947B5005EF24E0FF2208
:01712F00223D
:00000001FF
